:020000040800F2
:100000000080012007680008516700087D6800082B
:10001000556700085767000859670008000000008E
:100020000000000000000000000000005B67000806
:100030005D670008000000005F6700089529000860
:10004000636700086567000867670008696700085C
:100050006B6700086D6700086F670008716700082C
:1000600073670008756700087767000879670008FC
:100070007B6700087D6700087F67000881670008CC
:10008000836700088567000887670008896700089C
:100090008B6700088D6700088F670008916700086C
:1000A000936700089567000897670008996700083C
:1000B0009B6700089D6700089F670008A16700080C
:1000C000A3670008A5670008A7670008A9670008DC
:1000D000AB670008992A0008AF670008B1670008FD
:1000E000B3670008B5670008B7670008B96700087C
:1000F000BB670008BD670008BF670008C16700084C
:10010000C3670008C5670008C7670008C96700081B
:10011000CB670008CD670008CF670008D1670008EB
:10012000D3670008D5670008D7670008D9670008BB
:10013000DB670008DD670008DF670008E16700088B
:10014000E3670008E5670008E76700083D750008F9
:10015000EB670008ED670008EF670008F16700082B
:10016000F3670008F5670008F7670008F9670008FB
:10017000FB670008FD670008FF67000801680008CA
:0801800003680008056800088F
:1001880082B003468DF807309DF90730002B0CDB51
:100198009DF8073003F01F0205499DF907305B09F8
:1001A800012000FA02F241F8232000BF02B0704794
:0401B80000E100E082
:1001BC0082B0034600918DF807309DF90730002B73
:1001CC000ADB009BDAB20C499DF907301201D2B25E
:1001DC000B4483F800230BE0009BDAB207499DF82F
:1001EC00073003F00F03043B1201D2B20B441A7612
:1001FC0000BF02B0704700BF00E100E000ED00E07E
:10020C0000B583B00190019B013BB3F1807F01D31A
:10021C0001230FE0094A019B013B53600F214FF072
:10022C00FF30FFF7C5FF054B00229A60034B0722F6
:10023C001A600023184603B05DF804FB10E000E0E0
:10024C0000B583B07F4B9B6D7E4A43F08053936522
:10025C007C4BDB6C7B4A43F00103D364794BDB6C46
:10026C00784A43F00203D364764BDB6C754A43F057
:10027C000403D364734BDB6C724A43F00803D364FE
:10028C004FF0904300221A606F4B00221A606F4BA4
:10029C0000221A606E4B00221A604FF090436D4A98
:1002AC00DA60694B6C4ADA60684B6C4ADA60684B0E
:1002BC002022DA6000F0F8FC4FF090431B684FF0FE
:1002CC00904223F002031360604B1B685F4A43F0BB
:1002DC00010313605D4B1B685C4A43F0040313601D
:1002EC005A4B03229A614FF090431B684FF0904297
:1002FC0023F4006313604FF090431B684FF090425F
:10030C0043F480631360564B1B68564AA2FB0323CD
:10031C009B091846FFF774FF534B14221A60534B7A
:10032C0000221A60524B00221A60524B00221A60B3
:10033C00514B00221A60514B4FF47A721A60504B99
:10034C004FF47A721A604F4B00221A604E4B002207
:10035C001A604E4B00221A604D4B00221A604D4B16
:10036C0001221A604C4B00221A604C4B00221A607E
:10037C004B4B00221A604B4B00221A604A4B45F241
:10038C0055521A60484B4FF6FF729A60022000F0EB
:10039C0029FD454B02225A60022000F023FD424BFE
:1003AC004CF6CC421A60294BDB68284A43F05003C8
:1003BC00D360264BDB68254A23F0A003D3600220D0
:1003CC0000F010FD394B00221A60204B1B6903F022
:1003DC000403002B02D1354B01221A6001F010FDF1
:1003EC0002F028F8314B1B68002B0BD10A2000F0CF
:1003FC00F9FC4F2002F06CF96B2002F069F90D202A
:10040C0002F066F90A2000F0EDFC294B00221A607C
:10041C0002F0C6FB184B40F6B8321A6003E0164BDC
:10042C001B68002B04D0224B1B68002BF7D000E07C
:10043C0000BF06F08AFC184B00221A6000238DF8CE
:10044C00073042E000100240000400480008004859
:10045C00000C0048AAAA02A48AAAAAAAAAAAAAA616
:10046C000C000020D34D6210783100208C3100201C
:10047C007C3100209C3100206C3100208831002020
:10048C005C31002070310020483100207431002094
:10049C0090310020843100209431002098310020CC
:1004AC0068310020803100200030004040310020B5
:1004BC00443100209DF80730894A002122F813109E
:1004CC009DF8073001338DF807309DF80730112B5C
:1004DC00F0D901F007F9642000F084FC00F036FD3F
:1004EC00642000F07FFC00F031FD0A2000F07AFC63
:1004FC007C4B00221A607C4B1B6903F00803002B19
:10050C0002D1784BFF221A600A2000F06BFC774B6B
:10051C001B68002B05D1764B1B68002B01D004F017
:10052C00D5F802F0CBF90346ADF80430BDF8043031
:10053C00002B64D0BDF804308DF807306B4B1B6872
:10054C00002B57D16B4B1B68002B4DD16A4B1B6892
:10055C00042B06D1694B1B68002B02D0664B002282
:10056C001A609DF807302B2B0AD1634B1B68022BAA
:10057C0006D1614B03221A60604B4FF47A721A60F9
:10058C009DF807302B2B0AD15B4B1B68012B06D136
:10059C00594B02221A60594B4FF4C8721A609DF8DD
:1005AC0007302B2B0ED1544B1B68002B0AD1534B0D
:1005BC001B68002B06D1504B01221A604F4B4FF495
:1005CC00C8721A604A4B1B68002B18D19DF8073073
:1005DC00184603F003FE484B1B68002B0FD1474B0A
:1005EC004FF47A721A600AE09DF80730184603F04F
:1005FC00F5FD04E09DF80730184603F015FE404B5E
:10060C001B68002B83D003F043FC0346ADF8043089
:10061C00BDF80430002B3FF47AAFBDF804308DF8F0
:10062C000730324B1B68002B54D1334B1B68002B0B
:10063C007FF46DAF2F4B1B68042B06D1314B1B681D
:10064C00002B02D02B4B00221A609DF807302B2B6D
:10065C000AD1284B1B68022B06D1264B03221A60A9
:10066C00284B4FF47A721A609DF807302B2B0AD165
:10067C00204B1B68012B06D11E4B02221A60214B0A
:10068C004FF4C8721A609DF807302B2B0ED1194B02
:10069C001B68002B0AD11B4B1B68002B06D1154B7A
:1006AC0001221A60174B4FF4C8721A60104B1B686A
:1006BC00002B7FF42CAF9DF80730184602F008F899
:1006CC000C4B1B68002B7FF422AF0E4B4FF47A724D
:1006DC001A601CE79DF80730184601F0F9FF16E781
:1006EC00E430002094310020000800484031002004
:1006FC0074310020483100207031002088310020F6
:08070C00443100205C310020A3
:1007140082B00190019B013B102B00F2AC8201A23C
:1007240052F823F06D070008DB07000849080008A9
:100734009F0800080D0900087B090008E909000862
:100744001B0A0008410A0008710A0008970A0008F9
:10075400BD0A00082B0B00089B0B0008090C0008BD
:100764002F0C0008550C00084FF090431B684FF005
:10077400904223F0300313604FF09043DB684FF056
:10078400904223F02003D3604FF09043DB684FF096
:10079400904243F01003D360B24B5B8A1BB2002B30
:1007A40080F26B824FF090431B684FF0904243F00D
:1007B400300313604FF09043DB684FF0904223F016
:1007C4003003D3604FF09043DB6A4FF0904243F024
:1007D4000403D36251E24FF090431B684FF0904200
:1007E40023F0C00313604FF09043DB684FF0904256
:1007F40023F08003D3604FF09043DB684FF09042C6
:1008040043F04003D360974BDB8A1BB2002B80F28A
:1008140036824FF090431B684FF0904243F0C00380
:1008240013604FF09043DB684FF0904223F0C00315
:10083400D3604FF09043DB6A4FF0904243F00803DB
:10084400D3621CE2884B1B68874A23F003031360BE
:10085400854BDB68844A23F00203D360824BDB6858
:10086400814A43F00103D3607E4B5B8B1BB2002BA8
:1008740080F207827C4B1B687B4A43F003031360BE
:10088400794BDB68784A23F00303D360764BDB6A49
:10089400754A43F00103D362F3E14FF090431B68C0
:1008A4004FF0904223F4407313604FF09043DB68A1
:1008B4004FF0904223F40073D3604FF09043DB6811
:1008C4004FF0904243F48073D360664BDB8B1BB2D2
:1008D400002B80F2D8814FF090431B684FF0904278
:1008E40043F4407313604FF09043DB684FF0904241
:1008F40023F44073D3604FF09043DB6A4FF090428F
:1009040043F01003D362BEE14FF090431B684FF0F5
:10091400904223F00C0313604FF09043DB684FF0D8
:10092400904223F00803D3604FF09043DB684FF00C
:10093400904243F00403D3604A4B5B8C1BB2002B00
:1009440080F2A3814FF090431B684FF0904243F034
:100954000C0313604FF09043DB684FF0904223F098
:100964000C03D3604FF09043DB6A4FF0904243F0A6
:100974000203D36289E14FF090431B684FF0904229
:1009840023F0030313604FF09043DB684FF0904271
:1009940023F00203D3604FF09043DB684FF09042A2
:1009A40043F00103D3602F4BDB8C1BB2002B80F28E
:1009B4006E814FF090431B684FF0904243F0030365
:1009C40013604FF09043DB684FF0904223F0030331
:1009D400D3604FF09043DB6A4FF0904243F0010341
:1009E400D36254E14FF090431B684FF0904223F0E0
:1009F400404313604FF09043DB684FF0904223F084
:100A04000043D3604FF09043DB684FF0904243F0D3
:100A14008043D36042E1144B1B68134A23F44043E0
:100A24001360114BDB68104A23F40043D3600E4B70
:100A3400DB680D4A43F48043D3602FE10A4B1B6803
:100A4400094A23F0C0031360074BDB68064A23F00E
:100A5400C003D360044BDB68034A43F04003D36014
:100A64001CE100BF68300020000400488D4B1B6867
:100A74008C4A23F4406313608A4BDB68894A23F46D
:100A84004063D360874BDB68864A43F48063D3605A
:100A940004E1844B1B68834A23F440731360814B45
:100AA400DB68804A23F44073D3607E4BDB687D4A65
:100AB40043F48073D360F1E04FF090431B684FF030
:100AC400904223F4404313604FF09043DB684FF0AF
:100AD400904223F40043D3604FF09043DB684FF01F
:100AE400904243F48043D3606F4BDB8F1BB2002BE7
:100AF40080F2CF804FF090431B684FF0904243F454
:100B0400404313604FF09043DB684FF0904223F46E
:100B14004043D3604FF09043DB6A4FF0904243F080
:100B24008003D362B5E04FF090431B684FF09042CE
:100B340023F4405313604FF09043DB684FF090422E
:100B440023F40053D3604FF09043DB684FF090429E
:100B540043F48053D360544BB3F842301BB2002BA0
:100B640080F299804FF090431B684FF0904243F419
:100B7400405313604FF09043DB684FF0904223F4EE
:100B84004053D3604FF09043DB6A4FF0904243F000
:100B94004003D3627FE04FF090431B684FF09042D4
:100BA40023F4406313604FF09043DB684FF09042AE
:100BB40023F40063D3604FF09043DB684FF090421E
:100BC40043F48063D360384BB3F846301BB2002B38
:100BD40063DA4FF090431B684FF0904243F4406354
:100BE40013604FF09043DB684FF0904223F440636E
:100BF400D3604FF09043DB6A4FF0904243F0200300
:100C0400D3624AE0274B1B68264A23F4402313602F
:100C1400244BDB68234A23F44023D360214BDB6855
:100C2400204A43F48023D36038E01E4B1B681D4ADE
:100C340023F4403313601B4BDB681A4A23F440331C
:100C4400D360184BDB68174A43F48033D36025E044
:100C5400164B1B68154A23F040631360134BDB6883
:100C6400124A23F04063D360104BDB680F4A43F011
:100C74008063D36012E000BF10E000BF0EE000BF4D
:100C84000CE000BF0AE000BF08E000BF06E000BFC0
:100C940004E000BF02E000BF00E000BF00BF02B0FC
:100CA400704700BF00040048683000200008004876
:100CB400424B9B6D414A43F08053936500BF404BC8
:100CC4005B6903F48063002BF9D13D4B1B683C4AFC
:100CD40023F4806313603A4B1B68394A43F440732E
:100CE400136000BF364B5B6903F48063002BF9D1BA
:100CF400344B1B68334A43F4817313602F4B1B68D6
:100D04002E4A23F08073136000BF2C4B1B6803F042
:100D14000073002BF9D1294BD3F89030274A23F0E4
:100D24003D03C2F89030254BD3F89030234A43F06A
:100D34001803C2F89030214BD3F890301F4A43F087
:100D44000103C2F8903000BF1C4BD3F8903003F07D
:100D54000203002BF8D000BF184B1B6803F00203FA
:100D6400002BF9D0154B1B68144A23F0F0031360D1
:100D7400124B1B68114A43F0B00313600F4B1B68FE
:100D84000E4A43F00D03136000BF0C4B1B6803F0C5
:100D94000203002BF9D0094B9B68084A43F4105313
:100DA4009360064BD3F88830044A43F04063C2F89A
:100DB4008830054B054A1A6000BF70470010024096
:100DC40000700040002002400C000020006CDC0297
:100DD400044B4FF400329A61034BC8221A6000BFDF
:0C0DE400704700BF000800487C31002070
:100DF00082B00346ADF80630BDF80630054A1360F0
:100E000000BF044B1B68002BFBD100BF00BF02B02A
:080E1000704700BF9C31002077
:100E180008B5444B14221A60434B4AF6AA221A60BA
:100E2800424B1B68002B01D100F092F8404B1B6825
:100E3800002B02D13F4B01229A613F4B1B68002BCC
:100E480002D13C4B02229A613C4B1B6801333B4A5E
:100E580013603A4B1B68312B62D9384B00221A6059
:100E6800374B9B884FF6FF72934203D1354B0022D4
:100E78001A7004E0324B9B88DAB2324B1A702D4B51
:100E88001B6903F00403002B11D12F4B1B68002BA7
:100E98000DD101F05DFE2C4B01221A6001F0CCFA55
:100EA8004FF4FA70FFF7A0FF01F07CFE16E0214B2B
:100EB8001B6903F00403002B10D0234B1B68012B84
:100EC8000CD101F045FE204B00221A6001F0B4FA63
:100ED8004FF4FA70FFF788FF01F064FE134B1B68AC
:100EE800002B1AD1134B1B6903F00803002B06D102
:100EF800164B1B68002B02D1144BFF221A600D4BB6
:100F08001B6903F00803002B0AD0104B1B68002B49
:100F180006D00E4B00221A6002E00C4B00221A6029
:100F280000BF08BD78310020003000409831002013
:100F38008C310020000800487C310020303100202E
:100F480010300020BA3100204031002094310020B8
:100F580000B583B07A4B9B6803F00103002B01D1E5
:100F680000F0C2FB774B5B8A4FF6FF72934223D0A7
:100F7800744B5B8A1BB2002B10DA734B1B68002B77
:100F88000CD0072000F05EFB0346ADF80630BDF834
:100F980006301946012000F015FA0DE04FF0904395
:100FA8001B699BB203F00403ADF80430BDF80430AC
:100FB8001946012000F008FB624BDB8A4FF6FF72EE
:100FC800934223D05F4BDB8A1BB2002B10DA5E4BB7
:100FD8001B68002B0CD0082000F034FB0346ADF84A
:100FE8000630BDF806301946022000F0EBF90DE096
:100FF8004FF090431B699BB203F00803ADF804302F
:10100800BDF804301946022000F0DEFA4D4B5B8B28
:101018004FF6FF72934222D04A4B5B8B1BB2002BD8
:1010280010DA494B1B68002B0CD00F2000F00AFB8C
:101038000346ADF80630BDF806301946032000F027
:10104800C1F90CE0414B1B699BB203F00103ADF8F9
:101058000430BDF804301946032000F0B5FA394BC6
:10106800DB8B4FF6FF72934223D0364BDB8B1BB2E0
:10107800002B10DA344B1B68002B0CD0092000F031
:10108800E1FA0346ADF80630BDF8063019460420EB
:1010980000F098F90DE04FF090431B699BB203F004
:1010A8001003ADF80430BDF804301946042000F0F0
:1010B8008BFA244B5B8C4FF6FF72934223D0214B63
:1010C8005B8C1BB2002B10DA1F4B1B68002B0CD05B
:1010D800062000F0B7FA0346ADF80630BDF8063032
:1010E8001946052000F06EF90DE04FF090431B699A
:1010F8009BB203F00203ADF80430BDF80430194682
:10110800052000F061FA0F4BDB8C4FF6FF7293421B
:101118002CD00C4BDB8C1BB2002B19DA0A4B1B684A
:10112800002B15D0052000F08DFA0346ADF80630E7
:10113800BDF806301946062000F044F916E000BF55
:101148000000045068300020A0310020000400484E
:101158004FF090431B699BB203F00103ADF80430D4
:10116800BDF804301946062000F02EFA914B5B8D2D
:101178004FF6FF7293420FD04FF090431B699BB21A
:1011880023F4FF4323F07F03ADF80430BDF80430A7
:101198001946072000F018FA864BDB8D4FF6FF72D0
:1011A80093420CD0844B1B699BB203F08003ADF8CB
:1011B8000430BDF804301946082000F005FA7D4BCC
:1011C8005B8E4FF6FF7293420CD07B4B1B699BB230
:1011D80003F00803ADF80430BDF8043019460920BF
:1011E80000F0F2F9734BDB8E4FF6FF7293420CD08E
:1011F800714B1B699BB203F02003ADF80430BDF8B6
:10120800043019460A2000F0DFF96A4B5B8F4FF66D
:10121800FF7293420CD0684B1B699BB203F010031A
:10122800ADF80430BDF8043019460B2000F0CCF9B5
:10123800604BDB8F4FF6FF72934223D05D4BDB8F01
:101248001BB2002B10DA5D4B1B68002B0CD00C2056
:1012580000F0F8F90346ADF80630BDF80630194637
:101268000C2000F0AFF80DE04FF090431B699BB2E3
:1012780003F08003ADF80430BDF8043019460C20A3
:1012880000F0A2F94B4BB3F842304FF6FF7293428D
:1012980024D0484BB3F842301BB2002B10DA474B2E
:1012A8001B68002B0CD00B2000F0CCF90346ADF8DE
:1012B8000630BDF8063019460D2000F083F80DE021
:1012C8004FF090431B699BB203F04003ADF8043024
:1012D800BDF8043019460D2000F076F9354BB3F807
:1012E80046304FF6FF72934224D0324BB3F8463063
:1012F8001BB2002B10DA314B1B68002B0CD00A20D4
:1013080000F0A0F90346ADF80630BDF806301946DE
:101318000E2000F057F80DE04FF090431B699BB288
:1013280003F02003ADF80430BDF8043019460E2050
:1013380000F04AF91F4BB3F84A304FF6FF72934258
:101348000CD01D4B1B699BB203F40073ADF804303D
:10135800BDF8043019460F2000F036F9154BB3F8E4
:101368004E304FF6FF7293420CD0134B1B699BB261
:1013780003F48073ADF80430BDF80430194610202A
:1013880000F022F90B4BB3F852304FF6FF7293423C
:101398000CD00B4B1B699BB203F40053ADF804301F
:1013A800BDF804301946112000F00EF900BF03B053
:1013B8005DF804FB6830002000040048A0310020DC
:0413C80000080048D1
:1013CC0000B585B003460A468DF807301346ADF8D4
:1013DC0004309DF807305B005B00744A13440293A1
:1013EC00029B1B884FF6FF72934200F0D980029B40
:1013FC0002331B884FF6FF72934200F0D3806C4B84
:10140C00DB88ADF80E30029B1B88ADF80C30BDF8B4
:10141C000C3003F0F003002B04D0BDF80C301B098A
:10142C00ADF80C30BDF80C300E2B07D1029B0233FB
:10143C001B8803F47F43B3F5014F0DD0BDF8043086
:10144C005B09ADF80430BDF80E30002B04D0BDF8AC
:10145C000E30023BADF80E309DF80730554A32F88D
:10146C001330BDF804209A4200F09D809DF807309F
:10147C00514AD35C002B49D09DF807304D4A32F8C5
:10148C001330BDF804209A4216D29DF807304B4910
:10149C00BDF8042021F81320494B1B68002B04D005
:1014AC009DF80730184600F081F99DF80730414946
:1014BC00BDF8042021F81320BDF804209DF8073056
:1014CC003C4931F813301946BDF80E300B449A42A2
:1014DC0069DD9DF807303949BDF8042021F8132047
:1014EC00374B1B68002B04D09DF80730184600F0D2
:1014FC005DF99DF807302F49BDF8042021F8132021
:10150C009DF807302C4A0021D1544CE09DF807304F
:10151C00284A32F81330BDF804209A4216D99DF8A7
:10152C0007302649BDF8042021F81320244B1B68F2
:10153C00002B04D09DF80730184600F037F99DF8C1
:10154C0007301C49BDF8042021F81320BDF80420F5
:10155C009DF80730174931F813301946BDF80E3095
:10156C00CB1A9A421FDA9DF807301449BDF80420B3
:10157C0021F81320124B1B68002B04D09DF8073068
:10158C00184600F013F99DF807300A49BDF80420FD
:10159C0021F813209DF80730074AFF21D15402E0AF
:1015AC0000BF00E000BF05B05DF804FB1C3000205C
:1015BC0010300020C03000201C310020E43000200E
:0415CC009431002036
:1015D00000B583B003460A468DF807301346ADF8D0
:1015E00004309DF80730164A32F81330BDF8042055
:1015F0009A4207D09DF807301149BDF8042021F820
:10160000132018E09DF807300E4A32F81330BDF869
:1016100004209A420FD09DF807300A49BDF80420F3
:1016200021F81320084B1B68002B04D09DF80730CD
:10163000184600F0D9F900BF03B05DF804FB00BF05
:0C164000C0300020E43000209431002075
:10164C0086B003468DF807300023059300238DF8F0
:10165C0013301FE0224B40F2FF721A609DF80730E6
:10166C009A011F4B1A631E4B9B681D4A43F00403DF
:10167C00936000BF1A4B1B6803F00403002BF9D0D6
:10168C00174B1B6C059A134405939DF813300133CB
:10169C008DF813309DF81330412BDBD9059B03F0EB
:1016AC000F030393059B1B090593039B072B02D97F
:1016BC00059B01330593059B403B0593059BB3F1BB
:1016CC007F4F01D900230593059BB3F5805F02D3AF
:1016DC0040F6FF730593059B9BB2184606B0704706
:0416EC0000000450A6
:1016F00008B52B4BDB6C2A4A43F40053D364294BC7
:101700009B68284A23F000539360264B9B68254A28
:1017100043F0805393600220FFF76AFB214BD3F81C
:10172000B030204A1B0C1B04C2F8B0301E4B4FF4E3
:1017300000329A600220FFF75BFB1A4B1B68194AC4
:1017400043F001031360174B9B68164A43F00103F3
:10175000936000BF134B1B6803F00103002BF9D00B
:10176000104B1B680F4A43F0010313600D4B082216
:10177000DA600C4B0D4A5A610A4B0D4A9A61094BCB
:1017800000221A63074B00225A63064B00229A6319
:10179000044B0022DA63074BFF221A6000BF08BD2A
:1017A00000100240000004500003045000806D1B34
:0817B000DB800100A0310020E4
:1017B80000B587B003468DF807309DF807305B0009
:1017C8005B00834A13440393039B1B884FF6FF7205
:1017D800934200F0F580039B1B88DBB2ADF80A301A
:1017E800BDF80A30F32B00F2ED80BDF80A308DF811
:1017F80017309DF817300F2B0AD89DF817301B01AA
:101808005AB2744B1B785BB213435BB28DF8173036
:101818009DF817301B09DBB2ADF80A30039B023381
:101828000393039B1B88ADF80830BDF808304FF6CA
:10183800FF72934200F0C880674B1B68012B04D1EC
:101848009DF81730184605F09EFA9DF80730634A50
:1018580032F81330ADF81230BDF80A300E2B44D1EF
:10186800BDF8083003F47F43B3F5014F17D1BDF835
:101878001230DBB29B00DBB203F07C038DF816302C
:10188800BDF812305B099BB28DF81530BDF81230E7
:101898006FEA43436FEA5343ADF8123009E000237F
:1018A8008DF81630BDF81230DBB203F07F038DF8E7
:1018B8001530494B1B68012B0DD19DF81630184681
:1018C80005F061FA9DF8153003F07F03DBB2184686
:1018D80005F059FA79E0BDF812209DF807109DF837
:1018E8001730184600F064F96FE0BDF80A300B2B8A
:1018F80003D99DF81730F22B27D1039B1B88DBB245
:1019080003F07F038DF81630BDF81230DBB203F018
:101918007F038DF81530304B1B68012B0AD19DF8D9
:101928001630184605F02FFA9DF81530184605F0C0
:101938002AFA4AE09DF815309AB29DF807109DF8EA
:101948001730184600F034F93FE0BDF80A300C2B88
:1019580007D0BDF80A300D2B03D09DF81730F32BB4
:101968001BD1BDF81230DBB203F07F038DF81530C0
:10197800194B1B68012B05D19DF81530184605F049
:1019880002FA22E09DF815309AB29DF807109DF8EA
:101998001730184600F00CF917E00F4B1B68012BA5
:1019A80006D1002005F0EFF9002005F0ECF90CE075
:1019B8009DF8173000221946452000F0F9F804E098
:1019C80000BF02E000BF00E000BF07B05DF804FB05
:1019D8001C300020BA31002040310020E4300020C3
:1019E80000B587B003468DF807309DF807305B00D7
:1019F8005B006B4A13440493049B9A1C04921B8853
:101A0800DBB2ADF80E30BDF80E30F52B23D9BDF89A
:101A18000E30F92B1FD0BDF80E30FD2B1BD09DF8D2
:101A28000730604A32F81330002B40F0B5805E4B27
:101A38001B68012B06D1BDF80E30DBB2184605F045
:101A4800A2F9A9E0BDF80E209DF80730194600203C
:101A580000F0AEF8A0E0BDF80E308DF817309DF814
:101A680017300F2B0AD89DF817301B015AB24F4B6D
:101A78001B785BB213435BB28DF817304A4B1B6877
:101A8800012B04D19DF81730184605F07CF99DF814
:101A980017301B09DBB2ADF80E30BDF80E300E2B37
:101AA80003D100238DF8163006E0049B1B88DBB2B7
:101AB80003F07F038DF816309DF80730394A32F865
:101AC8001330002B03D000238DF8153008E0049B59
:101AD8001B881B0A9BB2DBB203F07F038DF815301D
:101AE800BDF80E300C2B07D0BDF80E300D2B03D0EF
:101AF8009DF81730F32B13D12B4B1B68012B05D105
:101B08009DF81530184605F03EF946E09DF8153069
:101B18009AB29DF807301946002000F049F83CE0D9
:101B2800BDF80E30082B03D9BDF80E300B2B07D9A2
:101B3800BDF80E300E2B03D09DF81730F22B18D1BC
:101B4800194B1B68012B0AD19DF81630184605F071
:101B58001AF99DF81530184605F015F91DE09DF89D
:101B680015309AB29DF807301946002000F020F889
:101B780013E00D4B1B68012B06D1002005F003F97B
:101B8800002005F000F908E09DF8173000221946FA
:101B9800452000F00DF800E000BF07B05DF804FB39
:101BA8001C300020E430002040310020BA310020F1
:101BB80000B585B003468DF807300B468DF8063022
:101BC8001346ADF804308D4A02AB92E80300186062
:101BD8000433198002330A0C1A70202000F090FD9B
:101BE8009DF80730002B48D1232000F089FD9DF88F
:101BF8000630112B03D1752000F082FD15E09DF809
:101C08000630092B0AD9312000F07AFD9DF80630FC
:101C18002633DBB2184600F073FD06E09DF8063067
:101C28003033DBB2184600F06BFD642000F068FD2D
:101C3800BDF80430002B03D1302000F061FDD5E061
:101C48006F4B1B68002B0FD0302000F059FD782017
:101C580000F056FDBDF80430DBB203F07F03DBB2C1
:101C6800184605F0ACF8C1E0BDF8043003F07F0376
:101C78009BB2184600F09EFDB8E09DF80730452B52
:101C88002ED102AB184605F03DFC232000F038FDAC
:101C98009DF80630112B03D1752000F031FD15E0B9
:101CA8009DF80630092B0AD9312000F029FD9DF84E
:101CB80006302633DBB2184600F022FD06E09DF818
:101CC80006303033DBB2184600F01AFD452000F02C
:101CD80017FD722000F014FD722000F011FD85E060
:101CE800232000F00DFD9DF80630112B03D175203F
:101CF80000F006FD15E09DF80630092B0AD93120C1
:101D080000F0FEFC9DF806302633DBB2184600F0E2
:101D1800F7FC06E09DF806303033DBB2184600F0D9
:101D2800EFFC612000F0ECFC9DF8073003F0F003B5
:101D3800E02B3FD1BDF90430002B1EDA682000F0FB
:101D4800DFFC2F4B1B68002B0ED0302000F0D8FC96
:101D5800782000F0D5FCBDF80430C3F30B039BB228
:101D6800184605F06AF841E0BDF80430C3F30B03E8
:101D78009BB2184600F01EFD38E0214B1B68002B73
:101D88000FD0302000F0BCFC782000F0B9FCBDF882
:101D98000430DBB203F07F03DBB2184605F00FF81E
:101DA80024E0BDF8043003F07F039BB2184600F02E
:101DB80001FD1BE0124B1B68002B0FD0302000F0F8
:101DC8009FFC782000F09CFCBDF80430DBB203F0E7
:101DD8007F03DBB2184604F0F2FF07E0BDF80430D9
:101DE80003F07F039BB2184600F0E4FC202000F0CB
:101DF80087FC00BF05B05DF804FB00BF487400080D
:041E08008431002001
:101E0C0000B585B0044B0293044B0193044B009333
:101E1C0000238DF80F301BE000780008683000209C
:101E2C0010300020029B1A88019B1A80029B1A8892
:101E3C00009B1A80019B02330193009B0233009399
:101E4C00029B023302939DF80F3001338DF80F3053
:101E5C009DF80F302B2BE5D9984B1B884FF6FF7252
:101E6C00934205D1954B0B221A80954B0B221A806D
:101E7C00924B5B884FF6FF72934205D18F4B1F221A
:101E8C005A808F4B1F225A808C4B9B884FF6FF72C7
:101E9C00934205D1894B00229A80894B00229A806B
:101EAC00864BDB884FF6FF72934205D1834B04229D
:101EBC00DA80834B0422DA80804B1B894FF6FF7249
:101ECC00934205D07D4B5B894FF6FF7293420BD149
:101EDC007A4B04221A81794B83225A81784B042243
:101EEC001A81774B83225A81744B9B894FF6FF7270
:101EFC00934205D0714BDB894FF6FF7293420BD1A5
:101F0C006E4B57229A816D4B4022DA816C4B5722D3
:101F1C009A816B4B4022DA81684B1B8A4FF6FF7219
:101F2C0093420ED1654B0B221A82644B1A8A644B76
:101F3C001A82624B44F201025A82614B44F2010252
:101F4C005A825E4B9B8A4FF6FF7293420ED15B4BCB
:101F5C000B229A82594B9A8A594B9A82574B44F2CC
:101F6C000202DA82564B44F20202DA82534B1B8B8A
:101F7C004FF6FF7293420ED1504B0B221A834F4BEC
:101F8C001A8B4F4B1A834D4B44F203025A834C4B22
:101F9C0044F203025A83494B9B8B4FF6FF729342D8
:101FAC000ED1464B0B229A83444B9A8B444B9A830B
:101FBC00424B44F20402DA83414B44F20402DA83CA
:101FCC003E4B1B8C4FF6FF7293420ED13B4B0E22B5
:101FDC001A843A4B1A8C3A4B1A84384B4FF4014200
:101FEC005A84374B4FF401425A84344B9B8C4FF636
:101FFC00FF7293420ED1314B0B229A842F4B9A8C49
:10200C002F4B9A842D4B44F20602DA842C4B44F26B
:10201C000602DA84294B1B8D4FF6FF7293420ED1C8
:10202C00264B0B221A85254B1A8D254B1A85234BD3
:10203C0044F207025A85224B44F207025A851F4B81
:10204C009B8D4FF6FF7293420ED11C4B0B229A853F
:10205C001A4B9A8D1A4B9A85184B44F20802DA8562
:10206C00174B44F20802DA85144B1B8E4FF6FF72A5
:10207C0093420ED1114B0B221A86104B1A8E104B19
:10208C001A860E4B44F209025A860D4B44F2090291
:10209C005A860A4B9B8E4FF6FF72934213D1074B15
:1020AC000B229A86054B9A8E054B9A86034B44F26B
:1020BC000A02DA86024B44F20A0203E0683000207E
:1020CC0010300020DA866A4B1B8F4FF6FF7293425A
:1020DC000ED1674B0B221A87654B1A8F654B1A87EB
:1020EC00634B44F20B025A87624B44F20B025A8741
:1020FC005F4B9B8F4FF6FF7293420ED15C4B0B22C2
:10210C009A875B4B9A8F5B4B9A87594B44F20C0224
:10211C00DA87584B44F20C02DA87554BB3F840304F
:10212C004FF6FF72934213D1514B0E22A3F840206D
:10213C004F4BB3F840204F4BA3F840204C4B4FF47F
:10214C000042A3F842204B4B4FF40042A3F842202C
:10215C00474BB3F844304FF6FF72934213D1444BC4
:10216C000B22A3F84420424BB3F84420414BA3F874
:10217C0044203F4B44F20E02A3F846203D4B44F260
:10218C000E02A3F846203A4BB3F848304FF6FF72D4
:10219C00934213D1364B0B22A3F84820344BB3F89F
:1021AC004820344BA3F84820314B44F20F02A3F8DB
:1021BC004A20304B44F20F02A3F84A202C4BB3F8C0
:1021CC004C304FF6FF72934213D1294B0B22A3F8DC
:1021DC004C20274BB3F84C20264BA3F84C20244B17
:1021EC0044F21002A3F84E20224B44F21002A3F842
:1021FC004E201F4BB3F850304FF6FF72934213D161
:10220C001B4B0B22A3F85020194BB3F85020194B41
:10221C00A3F85020164B44F21102A3F85220154B90
:10222C0044F21102A3F85220114BB3F854304FF67C
:10223C00FF72934207D10E4B0122A3F854200D4B91
:10224C000122A3F854200A4B9B88DAB20A4B1A706D
:10225C00074BB3F854301A46084B1A60084B00224F
:10226C001A6004F072FD00BF05B05DF804FB00BFFE
:10227C006830002010300020BA310020843100205A
:04228C00903100206D
:1022900000B585B000BF624B1B6903F48033002B8F
:1022A000F9D15F4B5B69002B05DA5D4B5D4A9A60A3
:1022B0005B4B5D4A9A6000BF594B1B6903F4803346
:1022C000002BF9D1564B594A5A61554B5B69544A18
:1022D00043F48033536100BF514B1B6903F48033D7
:1022E000002BF9D14E4B1B6903F00103002B06D0E4
:1022F0004B4B1B694A4A43F0010313610AE0484B08
:102300001B69184604F0E3FD212000F0E7F92120C5
:1023100000F0E4F9424B5B69414A23F00203536148
:10232000434B1B689AB2434BA3F85420424B029391
:10233000404B01933A4B5B69394A43F001035361C7
:1023400000238DF80F304DE0019B1B880093019B0B
:1023500002330193019B1B881B04009A13430093D3
:10236000019B02330193029B009A1A60029B043383
:102370000293019B1B880093019B02330193019BF5
:102380001B881B04009A13430093019B02330193A3
:10239000029B009A1A60029B0433029300BF204BF9
:1023A0001B6903F48033002BF9D11D4B1B6903F02B
:1023B0000103002B06D01A4B1B69194A43F0010395
:1023C00013610AE0164B1B69184604F080FD2120BA
:1023D00000F084F9212000F081F99DF80F300133DD
:1023E0008DF80F309DF80F30152BADD90C4B5B6974
:1023F0000B4A23F001035361094B5B69084A43F020
:10240000004353610A20FEF7F3FC0C4B1B6843F0BA
:102410007F430A4A136000BF05B05DF804FB00BFAC
:102420000020024023016745AB89EFCD7A0000010F
:1024300084310020683000200078000890310020AE
:1024400000B583B09D4B1B6E9C4A43F480431366DA
:102450004FF090431B684FF0904223F480131360B9
:10246000974B1B68964A23F4805313604FF09043B8
:102470001B684FF0904243F400131360904B1B68AD
:102480008F4A43F4005313604FF090435B6A4FF060
:10249000904223F4706353624FF090435B6A4FF0B5
:1024A000904243F4E0635362854B1B6A844A23F0F5
:1024B00070631362824B1B6A814A43F0E0631362CC
:1024C000804B814A1A60814B7F4A1A60804B1B689F
:1024D000002B70D17F4B1B88602B46D0602B61DCBA
:1024E000262B3FDC0B2B5DDB0B3B1B2B5AD801A2B1
:1024F00052F823F09D250008A5250008A525000811
:10250000A5250008A5250008A5250008A525000883
:10251000A525000875250008A5250008A5250008A3
:10252000A5250008A5250008A5250008A525000863
:10253000A5250008A5250008A5250008A525000853
:10254000A52500087F250008A5250008A525000869
:10255000A5250008A5250008A5250008A525000833
:1025600089250008392B14D01CE04FF41C63ADF80A
:1025700006301BE04FF49C63ADF8063016E04FF4D4
:102580004073ADF8063011E04FF41C73ADF806301F
:102590000CE04FF4D073ADF8063007E0D023ADF86F
:1025A000063003E0D023ADF8063000BF4A4ABDF83C
:1025B0000630D36071E0474B5B88602B47D0602BBF
:1025C00062DC262B40DC0B2B5EDB0B3B1B2B5BD832
:1025D00001A252F823F000BF8126000889260008D6
:1025E000892600088926000889260008892600080F
:1025F000892600088926000859260008892600082F
:1026000089260008892600088926000889260008EE
:1026100089260008892600088926000889260008DE
:1026200089260008892600086326000889260008F4
:1026300089260008892600088926000889260008BE
:10264000892600086D260008392B14D01CE04FF4B1
:102650001C63ADF806301CE04FF49C63ADF8063007
:1026600017E04FF44073ADF8063012E04FF41C73DE
:10267000ADF806300DE04FF4D073ADF8063008E049
:10268000D023ADF8063004E04FF44073ADF80630C7
:1026900000BF114ABDF80630D3600F4B4FF4003233
:1026A0005A600D4B00229A600B4B2D221A60252098
:1026B000FDF76AFD00BF03B05DF804FB00100240A7
:1026C0000004004864310020102000206031002008
:0C26D0004031002068300020003801403C
:1026DC0082B003468DF8073000BF074BDB6903F06F
:1026EC008003002BF9D0044B9DF8072092B21A8579
:0C26FC0000BF02B0704700BF0038014072
:1027080000B583B003468DF807300F4B1B68772B55
:1027180003D00D4B1B68002B04D19DF807301846D9
:10272800FFF7D8FF084B1B68FF2B03D0064B1B682D
:10273800002B04D19DF80730184601F051FD00BF69
:0C27480003B05DF804FB00BF74310020FA
:1027540000B585B003468DF807309DF80730303357
:102764008DF80F309DF80F30392B04D99DF80F30B8
:1027740007338DF80F300F4B1B68772B03D00D4BAD
:102784001B68002B04D19DF80F301846FFF7A4FFF7
:10279400084B1B68FF2B03D0064B1B68002B04D18E
:1027A4009DF80F30184601F01DFD00BF05B05DF81F
:0827B40004FB00BF743100209A
:1027BC0000B585B00346ADF80630BDF80630092BE0
:1027CC0065D9BDF80630632B44D9BDF80630B3F596
:1027DC007A7F1DD3BDF80630354AA2FB03239B0933
:1027EC009BB20393039B9BB21A465201D21A9200DE
:1027FC001344DB009BB2BDF80620D31AADF80630AB
:10280C00039BDBB23033DBB21846FFF777FF00E0F7
:10281C0000BFBDF80630274AA2FB03235B099BB21D
:10282C000393039B9BB21A46920013441A469100E1
:10283C001A460B4613449B009BB2BDF80620D31AD4
:10284C00ADF80630039BDBB23033DBB21846FFF732
:10285C0055FF00E000BFBDF80630174AA2FB03236A
:10286C00DB089BB20393039B9BB21A469200134462
:10287C005B009BB2BDF80620D31AADF80630039B63
:10288C00DBB23033DBB21846FFF738FF00E000BF95
:10289C00BDF80630DBB23033DBB21846FFF72EFF43
:1028AC002020FFF72BFF00BF05B05DF804FB00BF35
:0C28BC00D34D62101F85EB51CDCCCCCC6D
:1028C80000B583B0154B1B68002B01D1FEF7A0FAA9
:1028D800134B1A68134B1B689A421AD0104B1B688B
:1028E8005A1C0F490A601B7843F4004301930C4BB0
:1028F8001A680D4B1B689A4202D1094B0B4A1A60A1
:102908000B4B4FF480329A610A4BC8221A60019B24
:1029180000E00023184603B05DF804FB783100207E
:1029280060310020643100200800002010200020C1
:08293800000800488C3100206A
:1029400000B583B0124B1B68FF2B03D0104B1B68E4
:10295000002B07D101F0A2FA03460193002B01D00E
:10296000019B10E00A4B1B68772B03D0084B1B68B8
:10297000002B07D1FFF7A8FF03460193002B01D0DE
:10298000019B00E00023184603B05DF804FB00BF84
:04299000743100207E
:10299400364B1B68002B0AD0344B1B68B3F5004F31
:1029A40005D2324B1B68013B304A136002E02F4BC7
:1029B40000221A602E4B1B68002B04D02C4B1B6882
:1029C400013B2B4A13602B4B1B68002B04D0294B73
:1029D4001B68013B274A1360274B1B68002B04D05C
:1029E400254B1B68013B244A1360244B1B68002BB6
:1029F40004D0224B1B68013B204A1360204B1B6808
:102A0400002B05D01E4B1B68013B1D4A136010E0D0
:102A14001C4B1B68032B09D11A4BFF221A601A4B5B
:102A2400FF221A60194B77221A6002E0154B00222C
:102A34001A60174B1B68002B05D0154B1B68013B14
:102A4400134A136010E0104B1B68032B09D10D4B84
:102A5400FF221A600C4BFF221A600C4BFF221A60F3
:102A640002E0094B00221A6000BF70477831002051
:102A74008C3100207C3100209C3100206C310020FE
:102A8400883100207031002048310020743100204A
:042A94005C31002091
:102A98000D4BDB6903F02003002B12D00A4B9B8CF3
:102AA80098B20A4B1B685A1C08490A60C2B21A70CD
:102AB800064B1A68064B1B689A4202D1034B054A1B
:102AC8001A6000BF704700BF003801406431002021
:082AD80008000020102000207E
:102AE00082B003468DF807309DF90730002B0CDBD0
:102AF0009DF8073003F01F0205499DF907305B0977
:102B0000012000FA02F241F8232000BF02B0704712
:042B100000E100E000
:102B140082B003468DF807309DF90730002B13DB94
:102B24009DF8073003F01F0209499DF907305B093E
:102B3400012000FA02F2203341F82320BFF34F8F23
:102B440000BFBFF36F8F00BF00BF02B0704700BF6C
:042B540000E100E0BC
:102B580008B54FF090435B6A4FF0904223F47F230F
:102B680053624FF090431B684FF0904223F070730C
:102B780013604320FFF7CAFF084BDB6A074A43F498
:102B88008053D362054BDB6C044A23F48053D3642F
:102B9800034B00221A6000BF08BD00BF00100240AE
:042BA8004431002094
:102BAC0008B5734BDB6A724A43F48053D362704BA3
:102BBC00DB6A6F4A23F48053D3626D4BDB6C6C4A37
:102BCC0023F48053D3646B4B5B686A4A43F4806391
:102BDC0053604FF090435B6A4FF0904223F47F2395
:102BEC0053624FF090435B6A4FF0904243F42A23B8
:102BFC0053624FF090431B684FF0904223F0A07348
:102C0C0013604FF090431B684FF0904243F02073D9
:102C1C0013604FF090439B684FF0904223F0707319
:102C2C0093604FF090439B684FF0904243F0A07339
:102C3C0093604FF09043DB684FF0904223F0707339
:102C4C00D3604B4BDB6C4A4A43F48053D3644FF054
:102C5C00A0439B684FF0A04223F001039360464BC6
:102C6C0003221A6000BF4FF0A0431B69002BFADA55
:102C7C004FF0A0431B694FF0A04243F001031361D6
:102C8C000120FEF7AFF800BF4FF0A0431A693B4B91
:102C9C001340B3F1004FF7D10120FEF7A3F8364BE8
:102CAC005B68354A23F0020353600220FEF79AF862
:102CBC004FF0A0431B684FF0A04243F04003136059
:102CCC004FF0A0431B684FF0A04243F08003136009
:102CDC004FF0A0434FF480329A633220FEF782F813
:102CEC004FF0A043DB684FF0A04243F0804343F425
:102CFC001153D3603220FEF775F84FF0A0434FF01C
:102D0C00FF325A614FF0A0431D4A9A611D4B0022BD
:102D1C001A60194B00221A61174B00225A61164B8C
:102D2C000022DA6100F030F800BF4FF0A0435B697D
:102D3C0023F40053002BF8D000BF4FF0A0435B6985
:102D4C0023F48053002BF8D04FF0A0435B694FF075
:102D5C00A04243F440535361074B5B68064A43F46B
:102D6C00807353604320FFF7B5FE00BF08BD00BF62
:102D7C00001002400070004000080050010000806C
:082D8C00083C0080000E00501D
:102D94007C4B00221A607C4B03221A604FF0A04344
:102DA40080225A62794B7A4A1A607A4B7A4A1A60BC
:102DB4007A4B00221A607A4B1B68002B02D1794BA4
:102DC400794A1A604FF0A0431B694FF0A04243F0C8
:102DD4003003136100BF4FF0A0431B6903F03003BD
:102DE400002BF8D1714B00221A60714B1B68704A9A
:102DF40043F05B0313606F4B00221A606E4B4FF07D
:102E040000421A606D4B1B686C4A43F05B0313600D
:102E14006B4B6C4A1A606C4B6C4A1A606C4B1B68A7
:102E24006B4A43F05B0313606A4B00221A606A4BDF
:102E34004FF480021A60694B1B68684A43F05B03D5
:102E44001360674B00221A60664B4FF400021A604D
:102E5400654B1B68644A43F05B031360634B0022B9
:102E64001A60634B634A1A60634B1B68624A43F0FF
:102E74005B031360614B624A1A60494B1B68002B69
:102E840019D1604B604A1A60604B1B685F4A43F07B
:102E94005B0313605E4B00221A605E4B4FF44002EA
:102EA4001A605D4B1B685C4A43F05B0313605B4B29
:102EB40000221A6017E0534B00221A60534B1B6820
:102EC400524A43F05B031360514B00221A60514B8A
:102ED40000221A60504B1B684F4A43F05B03136097
:102EE4004E4B00221A60284B5B69274A43F00903C2
:102EF4005361254B1B69244A43F0190313614FF0B6
:102F0400A04300229A614FF0A0434FF0FF325A6170
:102F14004FF0A0439A694FF0A041414B13438B619A
:102F24004FF0A0439B684FF0A04243F081039360AD
:102F3400154B3C4ADA611A4B1B68002B05D1124B26
:102F4400DB69114A43F00803D3610F4B00225A6333
:102F5400354B00221A60354B00221A80344B354A17
:102F64001A60354B334A1A60344B354A1A60354B74
:102F7400334A1A60344B00221A70344B00221A7000
:102F840000BF704744310020000800502800005062
:102F9400800040000401005000014000080100507E
:102FA400403100200C010050800120000009005035
:102FB4000809005010090050000B0050080B005085
:102FC400100B0050400008602009005040004800E9
:102FD4002809005030090050200B0050280B0050E5
:102FE400300B00504009005048090050500900506F
:102FF400400B005040008800480B0050500B00501C
:1030040040000800600900501000CC00680900501E
:1030140070090050600B0050680B0050700B00509A
:1030240018380C000300050038310020A4310020BA
:1030340050310020100000204C3100205831002075
:103044001010002054310020AA310020AC3100209F
:1030540000B587B04FF0A0439B694FF0A04223F026
:1030640010039361924B05934FF0A0431B6A0393A3
:10307400039A904B13400293039B03F00F03002B1E
:103084003FD1029B029B8C4A93420BD1059B1B6848
:103094000293059B1B680193884B20221A60884B7E
:1030A40000221A80039B03F4F013B3F5402F28D1B8
:1030B400059B1B680293059B1B680193029BDAB274
:1030C400804B1A70029B1B0ADAB27F4B1A70029B68
:1030D4001B0C9AB27D4B1A807C4B1B881B0A9BB23B
:1030E400DAB27B4B1A70794B1B88DAB2794B1A70BF
:1030F400019B9AB2784B1A80019B1B0C9AB2774BB6
:103104001A80039A764B1340764A934240F0C48067
:10311400039B1B09DAB2744B1A7086E0059B1B688B
:103124000293724B1B68012B04D1029B184600F0DA
:1031340027FF7AE0029B8DF813306D4B1B685A1CF5
:103144006B490A609DF813201A70694B1A68694B21
:103154001B689A4202D1664B674A1A60624B1B781D
:10316400013BDAB2604B1A705F4B1B78002B6CD0BA
:10317400029B1B0A8DF813305D4B1B685A1C5C497B
:103184000A609DF813201A70594B1A68594B1B6832
:103194009A4202D1564B584A1A60534B1B78013B52
:1031A400DAB2514B1A70504B1B78002B4FD0029B54
:1031B4001B0C8DF813304E4B1B685A1C4C490A608B
:1031C4009DF813201A704A4B1A684A4B1B689A429E
:1031D40002D1474B484A1A60434B1B78013BDAB291
:1031E400414B1A70404B1B78002B32D0029B1B0EB4
:1031F4008DF813303E4B1B685A1C3D490A609DF8FC
:1032040013201A703A4B1A683A4B1B689A4202D13F
:10321400374B394A1A60344B1B78013BDAB2324BD4
:103224001A70314B1B78002B15D02F4B1B78194685
:103234002E4B1A6813465B00134499420CD92A4B4F
:103244001B78402B7FF66AAF06E000BF04E000BFA6
:1032540002E000BF00E000BF284B1A68244B1B6843
:103264009A4208D9224B1B6803F6FE72234B1B6853
:10327400D31A009305E01E4B1A68204B1B68D31A1F
:1032840000931F4B00221A60009B40F6B8729342D1
:1032940002D91B4BFF221A604FF0A0439B694FF0E9
:1032A400A04243F01003936100BF07B05DF804FB34
:1032B40000100050FF7F1E00700004003831002011
:1032C400A4310020AE310020AF3100201A3100209B
:1032D400B7310020B8310020A8310020A6310020E9
:1032E4000F001E0002000400AD3100204031002018
:1032F4005831002004000020101000205431002018
:043304003C31002038
:1033080000B583B0784B9B69DAB2774BDB69DBB2E7
:103318001340DBB28DF807309DF80730DBB203F0BD
:103328000103002B00F086806F4B1A696E4B5B6BB4
:10333800DB0103F08003134300936C4B1A68009B76
:1033480013400093009B03F08003002B13D0664BBF
:103358005B6B654A23F001035363654B1B68012BC4
:1033680007D0634B1B68062B03D0614B1B68A12B4E
:1033780001D100F07DFC009B03F00103002B49D034
:103388005A4B01221A605B4B1B88002B30D1584BDB
:103398001B68052B0BD0564B1B68092B07D0544BC9
:1033A8001B68222B03D0524B1B68202B10D1524B89
:1033B8001B68002B0CD1514B514A1A60514B524A91
:1033C8001A60524B1B68002B02D1514B514A1A60AC
:1033D800454B5B6B444A23F0010353634E4B4F4A02
:1033E8001A604F4B1B684E4A43F00443136011E0C8
:1033F800404B1B8843F400224A4B1A604A4B1B6817
:10340800494A43F004431360374B5B6B364A43F039
:1034180001035363009B03F01003002B02D0334BCE
:1034280010221A60009B03F00803002B02D02F4BD8
:1034380008221A609DF80730DBB203F00203002B64
:1034480000F0AD80284B1A69274B5B6B9B0103F09A
:10345800800313430093354B1A68009B1340009375
:10346800009B03F08003002B07D01F4B5B6B1E4AA9
:1034780023F00203536300F06BFC009B03F001038D
:10348800002B04D1009B03F01003002B7FD0009B7E
:1034980003F00103002B02D0244B01221A60244BB5
:1034A8001A68244B1B689A420CD1144B1B68134AA8
:1034B80043F0044313600C4B5B6B0B4A23F002038D
:1034C80053635CE01A4B1A681A4B1B689A4235D949
:1034D800184B1B6803F6FE72154B1B68D31A9AB279
:1034E800154B1A8032E000BF000800500809005050
:1034F80038310020A4310020443100202009005038
:1035080040804884400B005040808884403100202F
:10351800600900501080CC84100B005040000860F7
:10352800000B0050100900500009005028090050F5
:103538004C310020503100202E310020484B1A68B1
:10354800484B1B68D31A9AB2474B1A80464B1B88C4
:10355800402B02D9444B40221A80434B1B8843F42A
:103568000022424B1A60424B1B68414A43F0044315
:103578001360404B5B6B3F4A43F002035363009B6D
:1035880003F01003002B02D03B4B10221A60009B63
:1035980003F00803002B02D0374B08221A609DF86D
:1035A8000730DBB203F00803002B54D0314B1A6903
:1035B800304B5B6B1B0103F08003134300932F4BCD
:1035C8001A68009B13400093009B03F08003002BB4
:1035D80009D02B4B4FF400221A602A4B1B68294A4A
:1035E80043F004431360009B03F00103002B12D047
:1035F800234B4FF400221A60224B1B68214A43F0E8
:10360800044313601D4B01221A601A4B5B6B194A65
:1036180023F008035363009B03F01003002B12D020
:10362800174B4FF400221A60164B1B68154A43F0DB
:10363800044313600F4B5B6B0E4A23F0080353637C
:103648000E4B10221A60009B03F00803002B02D0D7
:103658000A4B08221A6000BF03B05DF804FB00BFE4
:10366800503100204C3100202E310020300900500C
:10367800200900500008005028090050680900502F
:083688007009005060090050B8
:1036900000B583B0774B9A69764BDB6913401B0CFE
:1036A000DBB28DF807309DF80730DBB203F0010381
:1036B000002B00F0AB80704B1B68DAB26D4B5B697E
:1036C000DBB21340DBB28DF806309DF80630DBB27A
:1036D00003F00103002B2AD0674B01221A60674BCD
:1036E000674A1A60674B1B68664A43F004431360DD
:1036F000654B1B78802B0CD1644B1B78002B08D1B9
:103700009DF80630DBB243F00803DBB28DF80630DB
:103710000DE05F4B1B68202B09D15E4B4FF400225C
:103720001A605D4B1B685C4A43F0044313609DF8CC
:103730000630DBB203F00803002B00F0978000F0A6
:10374000BBF8534B1B68052B1BD14A4B1B68534AD4
:10375000127812011146474A0B4313604D4B4FF448
:1037600000221A604C4B1B684B4A43F00443136021
:10377000414B08221A603F4B5B6B3E4A43F001030A
:103780005363434B1B68092B03D0414B1B68222B0F
:1037900012D1404B4FF400221A603F4B1B683E4A47
:1037A00043F004431360344B08221A60314B5B6BC7
:1037B000304A43F001035363354B1B68012B07D09C
:1037C000334B1B68062B03D0314B1B68A12B4DD10B
:1037D000334B1B88402B03D92E4B324A1A6005E02D
:1037E0002F4B1B8843F400222A4B1A602A4B1B687C
:1037F000294A43F0044313601F4B08221A601D4BF3
:103800005B6B1C4A43F0010353632FE09DF80730C4
:10381000DBB203F00403002B29D0234B1B68DAB280
:10382000144B5B69DBB21340DBB28DF806309DF8B8
:103830000630DBB203F00103002B18D01A4B012233
:103840001A601A4B174A1A60194B1B68002B06D1D5
:10385000184B1B68174A43F00443136007E0154BED
:103860001B68144A43F00043136000E000BF03B03C
:103870005DF804FB00080050080B0050100B0050CE
:1038800040000860000B0050AE310020AF31002036
:10389000383100201009005000090050B9310020D3
:1038A000A431002040000800480B0050500B00508D
:0838B0003C310020400B0050E8
:1038B80000B583B0914B00221A60914B1B78212BE5
:1038C80024D1904B1B78202B12D18F4B1B688E4A2A
:1038D80043F0080313608D4B8D4A1A608D4B1B68AB
:1038E8008C4A43F004431360844B20221A609AE107
:1038F800844B1B78222B06D1804B22221A60864BE0
:1039080000221A808FE100F019FA8CE17C4B1B78B9
:10391800A12B17D17B4B1B78212B13D1774BA122DD
:103928001A607D4B07221A807C4B1A887A4B1B88B9
:103938009A4203D2794B1A88774B1A80784B794A86
:103948001A6070E16E4B1B7803F06103002B06D000
:103958006B4B1B7803F06103012B40F06281694BCC
:103968001B78092B00F2568101A252F823F000BF00
:10397800A13900081D3C00081D3C00081D3C00083A
:103988001D3C0008C9390008E73900081D3C00083B
:103998001D3C0008EF3B0008584B01221A605E4BA3
:1039A80002221A805D4B1A885B4B1B889A4203D20D
:1039B8005A4B1A88584B1A80594B5B4A1A602FE1A8
:1039C8005A4B1B88DBB203F07F03DAB2584B1A70EC
:1039D8004A4B05221A60504B00221A8020E1474BBF
:1039E80006221A60534B1B78012B65D14A4B1222D1
:1039F8001A804A4B1A88484B1B889A4203D2474B75
:103A08001A88454B1A804C4B1B68012B03D1444B39
:103A18004A4A1A6002E0424B494A1A60494B0093ED
:103A28000023ADF806300EE03D4B1A68531C3C49A4
:103A38000B60009B591C009112781A70BDF8063073
:103A48000133ADF80630BDF80630112BECD93E4BEA
:103A58001A893D4B5B8913439AB23B4B9B891343AD
:103A68009AB2394BDB891343ADF80630BDF80630FE
:103A7800002B1DD0344B5B89DAB2324B1A72324BB1
:103A88001B89DAB22F4B5A722F4BDB89DAB22D4BD6
:103A98009A722D4B9B89DAB22A4BDA72264B1B6835
:103AA800012B05D1274B9B7A0233DAB2254B9A7248
:103AB8001B4B244A1A60B0E01E4B1B78022B49D1DD
:103AC8001D4B1B68012B06D1134B65221A80144B22
:103AD8001E4A1A6005E0104B43221A80104B1C4AFC
:103AE8001A600E4B1A880C4B1B889A4280F09580FE
:103AF8000A4B1A88084B1A808FE000BF3831002023
:103B0800AE310020AF310020080B0050100B0050E0
:103B180040000860000B0050A4310020A6310020AE
:103B2800343100201C740008406E00081A3100204F
:103B3800B9310020B731002040310020BC6E0008A8
:103B48007C6D00080831002068300020BC71000836
:103B5800D8730008354B1B78032B41D1344B1B78A5
:103B6800012B10D1334B18221A80334B1A88314B52
:103B78001B889A4203D2304B1A882E4B1A802F4B3F
:103B88002F4A1A6049E02A4B1B78022B10D1294B87
:103B980012221A80284B1A88264B1B889A4203D275
:103BA800254B1A88234B1A80244B264A1A6034E086
:103BB8001F4B1B78002B10D11E4B04221A801E4B62
:103BC8001A881C4B1B889A4203D21B4B1A88194B24
:103BD8001A801A4B1C4A1A601FE000F0AFF822E066
:103BE80000F0ACF819E0194B09221A60114B0022B9
:103BF8001A80174BFF221A60164B174A1A60174B88
:103C0800174A1A60174B1B68002B08D1164B174A26
:103C18001A6004E000F092F802E000BF03E000BF81
:103C280001E000F08BF803B05DF804FBB731002029
:103C3800B8310020A4310020A63100203431002002
:103C4800D0660008B46D0008CC6600083831002042
:103C5800443100202009005040804884400B005027
:103C68004080888440310020600900501080CC8456
:103C780084B02F4B1B88402B11D92E4B1B68039304
:103C88002C4B1B6840332B4A136040238DF80330BC
:103C9800274B1B88403B9AB2254B1A800AE0254BDC
:103CA8001B680393224B1B88DBB28DF80330204B33
:103CB80000221A809DF80330DBB20333002B00DAB0
:103CC80003339B10DBB28DF802301B4B02930023A9
:103CD8008DF801301FE0039B03331B781B061A463F
:103CE800039B02331B781B041343039A0132127897
:103CF80012021343039A127813430193019A029B09
:103D08001A60039B043303939DF80130DBB201333F
:103D1800DBB28DF801309DF80130DAB29DF802303F
:103D2800DBB29A42D7D300BF00BF04B0704700BFD0
:0C3D3800A43100203431002000100050A5
:103D4400034B1B68024A43F40013136000BF70471F
:043D5400000B005010
:103D580086B04A4B05934A4B1B6804937FE0494B56
:103D68001B681B780393474B1B680133454A136054
:103D7800444B1A68444B1B689A4202D1414B434A50
:103D88001A60434B1B88013B9AB2414B1A800023AF
:103D9800029300230193002300933D4B1B88002BC3
:103DA80017D0384B1B681B780293364B1B680133BE
:103DB800344A1360334B1A68334B1B689A4202D15A
:103DC800304B324A1A60324B1B88013B9AB2304B57
:103DD8001A802F4B1B88002B17D02A4B1B681B7887
:103DE8000193284B1B680133264A1360254B1A6838
:103DF800254B1B689A4202D1224B244A1A60244B55
:103E08001B88013B9AB2224B1A80214B1B88002B3E
:103E180017D01C4B1B681B7800931A4B1B68013387
:103E2800184A1360174B1A68174B1B689A4202D13D
:103E3800144B164A1A60164B1B88013B9AB2144B56
:103E48001A80009B1A06019B1B041A43029B1B0243
:103E58001A43039B13430493049A059B1A600C4B63
:103E68001B88002B7FF47BAF00BF054B1B68402BE2
:103E7800FBD100BF00BF06B0704700BF0020005054
:103E8800380900504C3100200000002010000020AC
:043E98002E310020A7
:103E9C0000B583B0304B1B68002B01D1FCF7B6FF8B
:103EAC002E4B1B68002B01D1002350E02C4B1A68C1
:103EBC002C4B1B689A4249D0FCF786FF284B1B6899
:103ECC005A1C27490A601B781BB26FEA43436FEAFE
:103EDC0053431BB29BB2ADF80630214B1A68224BF0
:103EEC001B689A4202D11E4B204A1A601C4B1A685E
:103EFC001C4B1B689A420CD91A4B1B681A46184B60
:103F0C001B68D31A9BB203F6FE739BB2ADF8043058
:103F1C0008E0144B1B681A46114B1B68D31A9BB252
:103F2C00ADF80430BDF804309BB240F6B772934242
:103F3C0008D80F4B00221A600E4B1B680D4A43F039
:103F4C0004431360BDF806309BB200E00023184612
:103F5C0003B05DF804FB00BF783100204431002031
:103F6C005431002058310020040000201010002093
:083F7C003C310020400B005015
:103F840000B585B00190019B8DF80F30904B1B78E4
:103F9400013BDAB28E4B1A708D4B1B78002B01D18A
:103FA400002311E1019B1B0A8DF80E30884B1B780E
:103FB400013BDAB2864B1A70854B1B78002B01D17A
:103FC400002301E1019B1B0C8DF80D30804B1B7805
:103FD400013BDAB27E4B1A707D4B1B78002B01D16A
:103FE4000023F1E0019B1B0E8DF80C30784B1B78FD
:103FF400013BDAB2764B1A709DF80F300F2B01D9C2
:104004000023E1E09DF80F30012B01D80023DBE011
:10401400FCF7DEFE9DF80F30052B03D09DF80F3022
:104024000F2B15D16B4B00221A706B4B1B685A1C5B
:1040340069490A609DF80E201A70674B1A68674B2D
:104044001B689A4202D1644B654A1A600123BBE0A3
:104054009DF80F300C2B03D09DF80F300D2B2DD174
:104064005C4B1B789DF80E209A4214D05A4B1B6867
:104074005A1C59490A609DF80E201A70564B1A684A
:10408400564B1B689A4202D1534B554A1A60514A07
:104094009DF80E301370504B1B685A1C4E490A6031
:1040A4009DF80D201A704C4B1A684C4B1B689A42B1
:1040B40002D1494B4A4A1A60012385E09DF80F302A
:1040C400022B03D09DF80F30062B26D1414B002242
:1040D4001A70414B1B685A1C3F490A609DF80E2018
:1040E4001A703D4B1A683D4B1B689A4202D13A4BF9
:1040F4003B4A1A60384B1B685A1C37490A609DF8C2
:104104000D201A70344B1A68344B1B689A4202D142
:10411400314B334A1A60012356E09DF80F30072BC8
:1041240014D82C4B00221A702B4B1B685A1C2A499A
:104134000A609DF80E201A70274B1A68274B1B68DB
:104144009A421ED1244B264A1A601AE0214B1B784E
:104154009DF80E209A4214D01F4B1B685A1C1E490E
:104164000A609DF80E201A701B4B1A681B4B1B68C3
:104174009A4202D1184B1A4A1A60164A9DF80E3018
:104184001370154B1B685A1C13490A609DF80D20C7
:104194001A70114B1A68114B1B689A4202D10E4BCC
:1041A4000F4A1A600C4B1B685A1C0B490A609DF895
:1041B4000C201A70084B1A68084B1B689A4202D1EB
:1041C400054B074A1A600123184605B05DF804FB45
:1041D400AD310020AC310020583100200400002013
:0441E4001010002097
:1041E80082B003468DF807300C4B1B68002B11D0AA
:1041F8000B4B1B685A1C0A490A609DF807201A7065
:10420800074B1A68074B1B689A4204D1044B064AAD
:104218001A6000E000BF02B0704700BF44310020C0
:0C42280050310020000000201000002099
:1042340084B003468DF80730A74B1B780133DAB2FC
:10424400A54B1A709DF90730002B80F2EF809DF882
:104254000730F72B02D0A04B01221A709DF80730CB
:10426400F02B0FD19D4BF0221A709D4BFF221A7038
:104274009C4B00221A709C4B00221A709B4B00220C
:104284001A700BE29DF80730F72B40F08780924BB1
:104294001B78012B35D1964B05221A708F4BF722D0
:1042A4001A70944B00221A70934B00221A708C4B94
:1042B40000221A708B4B00221A708B4B00221A704A
:1042C4008A4B1B78002B0CD0844BF7221A70894B35
:1042D40000221A70884B00221A70844B00221A7034
:1042E40084E17F4B00221A707B4B00221A707D4BB5
:1042F40000221A707C4B00221A707C4B00221A7028
:10430400CCE1754B1B78022B21D1794B06221A7014
:10431400724B1B78F02B03D0764B1A786F4B1A70C4
:10432400744B1A786D4B1A70724BF7221A70724BD9
:1043340000221A706A4B00221A706A4B00221A700B
:10434400694B00221A70694B00221A704EE1684BC7
:1043540007221A70614B1B78F02B07D1634B1B7833
:10436400002B03D1644BF7221A700AE0614B1A78D0
:104374005A4B1A70604B1A785E4B1A705E4BF722D8
:104384001A70574B00221A70564B00221A70564B63
:1043940000221A70554B00221A7027E14F4A9DF8EB
:1043A400073013704D4B1B78F32B0CD84C4BFF226A
:1043B4001A704C4B00221A704B4B00221A704B4B54
:1043C40000221A706AE1454B1B78F42B0BD0434B47
:1043D4001B78F52B07D0414B1B78F92B03D03F4BAF
:1043E4001B78FD2B0CD13E4B00221A703D4B002252
:1043F4001A703D4B00221A703C4B00221A704DE19A
:104404003B4B05221A703B4B00221A703A4B002298
:104414001A70334B00221A70324B00221A70324B3E
:1044240000221A70314B00221A70DFE02B4B1B78EC
:1044340023F00F038DF80B30294B1B78002B0CD184
:10444400254B00221A70274B00221A70264B00229B
:104454001A70264B00221A7020E1224B1B78002B85
:1044640050D1244A9DF807301370234B00221A7050
:104474001A4B1B78F12B03D0184B1B78F32B0FD15D
:104484001B4B02221A70164B00221A70154B002285
:104494001A70154B00221A70144B00221A70A5E0F2
:1044A4009DF80B30C02B03D09DF80B30D02B25D1B9
:1044B4009DF80B301B09DAB20D4B1A70084BFF2222
:1044C4001A70084B00221A70074B00221A70074B0F
:1044D40000221A708AE000BFAA310020B231002005
:1044E400B1310020B6310020B5310020AB310020BD
:1044F400B0310020B4310020B3310020684BFF22DA
:104504001A70CBE0674B1B78002B0CD1664B002252
:104514001A70634B00221A70644B00221A70644BA9
:1045240000221A70BAE0614B1B78002B43D1614A18
:104534009DF8073013705E4B1B78002B03D05B4B48
:10454400FF221A70AAE05C4B1B78F22B0FD15B4B55
:1045540003221A70534B00221A70514B00221A7016
:10456400524B00221A70524B00221A703EE0524BFA
:104574001B78F02B0FD1514B04221A704C4BFF22A5
:104584001A70484BFF221A70454B00221A70474B91
:1045940000221A702AE09DF80B301B09DAB2474B4F
:1045A4001A70404BFF221A703D4B00221A703F4B89
:1045B40000221A701AE0424B1A783F4B1A703D4B96
:1045C4001A783F4B1A703B4A9DF8073013703B4BE7
:1045D40004221A70364BFF221A70324BFF221A70D3
:1045E4002F4B00221A70314B00221A70354B1B6876
:1045F400002B52D0344B1B680393039B5A1C039229
:104604002E4A12781A70314B1B68039A9A4201D1D0
:104614002F4B0393039B5A1C0392274A12781A7058
:104624002A4B1B68039A9A4201D1294B0393039B9B
:104634005A1C0392224A12781A70244B1B68039A5C
:104644009A4201D1224B0393039B5A1C0392194AA9
:1046540012781A701D4B1B68039A9A4201D11C4BA5
:104664000393194A039B13600F4B00221A700C4BDF
:1046740000221A700D4B00221A70104B1B78072B66
:1046840003D80E4B1B78042B03D10B4B1B78F02B58
:1046940004D9044B00221A7000E000BF04B0704734
:1046A400B6310020B1310020AA310020B5310020FC
:1046B400AB310020B3310020B2310020B0310020F2
:1046C400B43100204431002050310020000000208B
:0446D40010000020B2
:1046D80030B5B9B0D64B26AC1D460FCD0FC40FCDA3
:1046E8000FC40FCD0FC495E80F0084E80F00D14B1D
:1046F8001EAC1D460FCD0FC495E80F0007C42380DC
:10470800CD4B16AC1D460FCD0FC495E80F0007C45E
:104718002370CA4B12AC0FCB07C42370C84B08AC2C
:104728001D460FCD0FC40FCD0FC495E8030084E8D4
:104738000300C44B04AC0FCB84E80F00C24B6C469B
:104748000FCB07C4238002341B0C237002F031FC0A
:10475800BE4802F0D7FE3320FDF7D2FF2E20FDF72A
:10476800CFFF3620FDF7CCFFB94802F0CBFE4FF45F
:104778007A70FCF739FB00238DF8DF3002F019FC62
:104788004320FDF7BDFF4D20FDF7BAFF4420FDF79C
:10479800B7FF3E20FDF7B4FF00BFFEF7CDF8034694
:1047A800ADF8DC30BDF8DC30002BF6D0BDF8DC30DD
:1047B8008DF8DF309DF8DF30202BEDD09DF8DF300D
:1047C8000A2B00D1E8E79DF8DF30602B08D99DF867
:1047D800DF307A2B04D89DF8DF30203B8DF8DF30AE
:1047E8009DF8DF30302B14D99DF8DF30392B10D8E5
:1047F8006B46184602F086FE9DF8DF301846FDF736
:104808007FFF9DF8DF30312B0ED03A20FDF778FF7F
:104818000AE09DF8DF301846FDF772FF3A20FDF7F1
:104828006FFF2020FDF76CFF9DF8DF300D3B712BEB
:1048380000F2818201A252F823F000BF374D000830
:104848003F4D00083F4D00083F4D00083F4D000810
:104858003F4D00083F4D00083F4D00083F4D000800
:104868003F4D00083F4D00083F4D00083F4D0008F0
:104878003F4D00083F4D00083F4D00083F4D0008E0
:104888003F4D00083F4D00083F4D00080D4A000805
:104898003F4D00083F4D00083F4D00083F4D0008C0
:1048A8003F4D00083F4D00083F4D00083F4D0008B0
:1048B8003F4D00083F4D00083F4D00083F4D0008A0
:1048C8003F4D00083F4D00083F4D0008854A00084D
:1048D800E14A0008E94A0008F14A0008F94A0008D4
:1048E800014B0008094B0008114B0008194B000840
:1048F8003F4D00083F4D00083F4D00083F4D000860
:104908003F4D0008134A0008294B00083F4D000896
:104918001F4A00082B4A00085D4A0008294C000875
:104928003F4D00083F4D0008314A00083F4D000840
:104938003F4D00083F4D00083F4D0008254A00083C
:104948003F4D00083F4D00083F4D00083F4D00080F
:104958003F4D00083F4D00083F4D0008214B00081F
:10496800194A00083F4D0008714A00083F4D0008E9
:104978003F4D00083F4D00083F4D00083F4D0008DF
:104988003F4D00083F4D00083F4D00083F4D0008CF
:104998003F4D00083F4D00083F4D00083F4D0008BF
:1049A8003F4D00083F4D00083F4D00083F4D0008AF
:1049B8003F4D00083F4D00083F4D00083F4D00089F
:1049C8003F4D00083F4D00083F4D00083F4D00088F
:1049D8003F4D00083F4D00083F4D00083F4D00087F
:1049E8003F4D00083F4D00083F4D00083F4D00086F
:1049F8003F4D00083F4D00083F4D00083F4D00085F
:104A0800AB4B000801F0D4F999E101F09DF896E16B
:104A180000F0AAF993E100F0BDFA90E100F0EEFB96
:104A28008DE100F0F9FC8AE100F088FD87E100BF24
:104A380094680008D4680008F4680008146900083D
:104A4800246900084C6900085C690008486D000882
:104A5800B4660008BB4B00221A60BB4802F052FD46
:104A6800BA4802F04FFD6AE1B64B01221A60B64817
:104A780002F048FDB64802F045FD60E102F03FFC57
:104A880003468DF8DB309DF8DB303F2B03D13F2008
:104A9800FDF736FE53E19DF8DB300D2B06D13A20A9
:104AA800FDF72EFE012000F095FD48E19DF8DB3072
:104AB800062B03D93F20FDF723FE40E13A20FDF7FE
:104AC8001FFE9DF8DB300A338DF8DB309DF8DB30B4
:104AD800184600F07FFD32E1022000F07BFD2EE158
:104AE800032000F077FD2AE1042000F073FD26E1A1
:104AF800052000F06FFD22E1062000F06BFD1EE1AD
:104B0800072000F067FD1AE1082000F063FD16E1B8
:104B1800092000F05FFD12E1112000F05BFD0EE1BD
:104B28000D20FDF7EDFD3E20FDF7EAFD4FF49670F0
:104B3800FCF75AF9FDF700FF0346002B05D03F208C
:104B4800FDF7DEFD2020FDF7DBFD08AB184602F07F
:104B5800D9FCFDF7F1FE0346ADF8DC30BDF8DC30DA
:104B6800002BF6D0BDF8DC3048F24002934213D156
:104B7800FDF748F902F0EBF82020FDF7C1FD6F20A2
:104B8800FDF7BEFD6B20FDF7BBFD2020FDF7B8FD4E
:104B9800704B00221A60D2E004AB184602F0B2FC57
:104BA800CDE00D20FDF7ACFD3E20FDF7A9FD4FF44B
:104BB8009670FCF719F9FDF7BFFE0346002B05D0E8
:104BC8003F20FDF79DFD2020FDF79AFD16AB184606
:104BD80002F098FCFDF7B0FE0346ADF8DC30BDF8F6
:104BE800DC30002BF6D0BDF8DC3048F27C02934272
:104BF80011D1FDF749FB2020FDF782FD6F20FDF75D
:104C08007FFD6B20FDF77CFD2020FDF779FD514BE2
:104C180000221A6093E012AB184602F073FC8EE093
:104C28004C4B1B6823F07F43002B65D04A4B012275
:104C38001A6026AB184602F065FC02F0BAF91EAB02
:104C4800184602F05FFC02F0B4F93E20FDF758FD6B
:104C580000BFFDF771FE0346ADF8DC30BDF8DC306F
:104C6800002BF6D0BDF8DC3048F21B02934203D18A
:104C7800394B00221A6062E0BDF8DC3048F27C0251
:104C8800934235D14FF49670FCF7AEF8FDF754FE19
:104C98000346002B05D03F20FDF732FD2020FDF70D
:104CA8002FFD16AB184602F02DFCFDF745FE034616
:104CB800ADF8DC30BDF8DC30002BF6D0BDF8DC30C8
:104CC80048F27C0293420ED1FDF7DEFA2020FDF770
:104CD80017FD6F20FDF714FD6B20FDF711FD202057
:104CE800FDF70EFD08E012AB184602F00BFC03E0DE
:104CF80012AB184602F006FC4520FDF701FD7820AE
:104D0800FDF7FEFC6920FDF7FBFC7420FDF7F8FCBD
:104D180002F04FF9114B00221A60114B00221A6061
:104D2800104B00221A600C4B00221A6008E00D207C
:104D3800FDF7E6FC03E03F20FDF7E2FC00BF1DE5C0
:104D480039B030BD84310020386700084467000856
:104D58004C67000890310020983100207431002001
:084D68007031002048310020E9
:104D700030B595B0834B09AC1D460FCD0FC40FCD98
:104D80000FC42B682370804B6C461D460FCD0FC49B
:104D90000FCD0FC42B6823707C4B01221A607C4B13
:104DA00000221A6002F009F909AB184602F0AEFBC6
:104DB000002002F036FA03468DF847309DF8473060
:104DC000EE2B03D1714B00221A60D8E09DF84730DA
:104DD000ADF84E30002002F024FA03468DF847303B
:104DE0009DF84730EE2B03D1684B00221A60C6E0D5
:104DF000BDF84E301B019AB29DF847309BB2134468
:104E0000ADF84E30002002F00CFA03468DF8473022
:104E10009DF84730EE2B03D15C4B00221A60AEE0C8
:104E20009DF84730ADF84C30002002F0FAF9034607
:104E30008DF847309DF84730EE2B03D1534B0022BD
:104E40001A609CE0BDF84C301B019AB29DF84730C7
:104E50009BB21344ADF84C30BDF84E20BDF84C3039
:104E600013439BB2002B07D14FF6FF73ADF84E30C2
:104E70004FF6FF73ADF84C3002F09FF86B461846C2
:104E800002F044FB002002F0CCF903468DF84730D5
:104E90009DF84730EE2B03D13C4B00221A606EE0A8
:104EA0009DF84730ADF84A30002002F0BAF90346C9
:104EB0008DF847309DF84730EE2B03D1334B00225D
:104EC0001A605CE0BDF84A301B019AB29DF8473089
:104ED0009BB21344ADF84A30002002F0A2F9034619
:104EE0008DF847309DF84730EE2B03D1274B002239
:104EF0001A6044E09DF84730ADF84830002002F0D9
:104F000090F903468DF847309DF84730EE2B03D1DA
:104F10001E4B00221A6032E0BDF848301B019AB2E5
:104F20009DF847309BB21344ADF84830BDF84A2095
:104F3000BDF8483013439BB2002B07D14FF6FF73E7
:104F4000ADF84A304FF6FF73ADF84830114ABDF85E
:104F50004E3013810F4ABDF84C3053810D4ABDF8D5
:104F60004A3093810B4ABDF84830D3810A4B1B6805
:104F700043F47F43084A1360044B00221A6015B0C3
:104F800030BD00BF6C6900089069000898310020AE
:0C4F900094310020683000209031002097
:104F9C0030B58DB0944B01AC1D460FCD0FC40FCD69
:104FAC000FC495E8030020600434218002340B0CFC
:104FBC0023708E4B01221A6001F0F9FF01AB1846E9
:104FCC0002F09EFA02F099F903468DF82F309DF805
:104FDC002F303F2B03D1854B00221A6001E19DF845
:104FEC002F308DF82E309DF82F30002B0FD09DF8E0
:104FFC002F30042B0BD09DF82F30062B07D09DF8AB
:10500C002F30072B03D09DF82F30082B06D13F20D3
:10501C00FDF774FB754B00221A60E2E002F06DF9AB
:10502C0003468DF82F309DF82F303F2B03D16F4B5B
:10503C0000221A60D5E09DF82E301A4692001344D7
:10504C005B00DAB29DF82F3013448DF82E309DF8AA
:10505C002E30392B68DC0B2BC0F2B1800B3B2E2B86
:10506C0000F2AD8001A252F823F000BF9751000866
:10507C00CB510008CB510008CB510008CB51000894
:10508C00CB510008CB510008CB5100084751000808
:10509C00CB510008CB510008CB510008B15100088E
:1050AC00CB510008CB510008CB510008CB51000864
:1050BC00CB510008CB510008CB5100085B510008C4
:1050CC00CB510008CB510008CB510008CB51000844
:1050DC00CB510008CB5100086F510008CB51000890
:1050EC00CB510008CB510008CB510008CB51000824
:1050FC00CB510008CB510008CB510008CB51000814
:10510C00CB510008CB510008CB510008CB51000803
:10511C00CB510008CB510008CB510008CB510008F3
:10512C00CB51000883510008602B48D13020FDF78B
:10513C00E5FA3020FDF7E2FA48E03220FDF7DEFA1E
:10514C003020FDF7DBFA3020FDF7D8FA3EE03220B4
:10515C00FDF7D4FA3520FDF7D1FA3020FDF7CEFA61
:10516C0034E03420FDF7CAFA3020FDF7C7FA3020BE
:10517C00FDF7C4FA2AE03220FDF7C0FA3020FDF723
:10518C00BDFA3020FDF7BAFA20E03520FDF7B6FA6B
:10519C003220FDF7B3FA3020FDF7B0FA3020FDF7DE
:1051AC00ADFA13E03020FDF7A9FA3420FDF7A6FA8A
:1051BC003020FDF7A3FA3020FDF7A0FA06E03F20DF
:1051CC00FDF79CFA094B00221A600AE09DF82E307C
:1051DC009AB2074B1A80074BFF221A60034B00222E
:1051EC001A600DB030BD00BFB469000898310020C2
:0851FC00683000209031002012
:1052040030B58DB0804B01AC1D460FCD0FC40FCD12
:105214000FC495E8030084E803007C4B01221A6064
:1052240001F0C9FE01AB184602F06EF902F069F80C
:1052340003468DF82F309DF82F303F2B03D1734B4D
:1052440000221A60DDE09DF82F308DF82E309DF895
:105254002F30002B13D09DF82F30022B0FD09DF848
:105264002F30042B0BD09DF82F30062B07D09DF840
:105274002F30072B03D09DF82F30082B06D13F2069
:10528400FDF740FA614B00221A60BAE002F039F8E7
:1052940003468DF82F309DF82F303F2B03D15B4B05
:1052A40000221A60ADE09DF82E301A469200134495
:1052B4005B00DAB29DF82F3013448DF82E309DF840
:1052C4002E30602B47D0602B00F38180262B3FDCEF
:1052D4000B2B7CDB0B3B1B2B79D801A252F823F060
:1052E400B9530008D3530008D3530008D35300081C
:1052F400D3530008D3530008D3530008D3530008F2
:1053040069530008D3530008D3530008D35300084B
:10531400D3530008D3530008D3530008D3530008D1
:10532400D3530008D3530008D3530008D3530008C1
:105334007D530008D3530008D3530008D353000807
:10534400D3530008D3530008D353000891530008E3
:10535400392B25D03BE03020FDF7D4F93020FDF780
:10536400D1F93BE03220FDF7CDF93020FDF7CAF941
:105374003020FDF7C7F931E03220FDF7C3F93520BD
:10538400FDF7C0F93020FDF7BDF927E03420FDF723
:10539400B9F93020FDF7B6F93020FDF7B3F91DE077
:1053A4003220FDF7AFF93020FDF7ACF93020FDF7DE
:1053B400A9F913E03520FDF7A5F93220FDF7A2F98C
:1053C4003020FDF79FF93020FDF79CF906E03F20DF
:1053D400FDF798F90D4B00221A6012E09DF82E306B
:1053E4009AB20B4B5A809DF82E309AB2094B5A80D0
:1053F400094B1B6843F47F03074A1360034B0022E5
:105404001A600DB030BD00BFDC690008983100207F
:0C54140068300020103000209031002093
:1054200030B589B0424B6C461D460FCD0FC495E890
:105430000F0007C423803F4B01221A6001F0BDFD1D
:105440006B46184602F062F801F05DFF03468DF8E6
:105450001E309DF81E303F2B03D1364B00221A60C0
:1054600064E09DF81E300A2B03D09DF81E300D2BF2
:1054700006D13F20FDF748F92E4B00221A6055E077
:105480009DF81E308DF81F3001F03DFF03468DF86A
:105490001E309DF81E303F2B03D1264B00221A6090
:1054A00044E09DF81E300D2B0ED09DF81F30DB0020
:1054B000DAB29DF81F305B00DBB21344DAB29DF81C
:1054C0001E3013448DF81F309DF81F30013B8DF8BE
:1054D0001F309DF81F300F2B15D92020FDF714F930
:1054E0003120FDF711F92D20FDF70EF93120FDF7E0
:1054F0000BF93620FDF708F92120FDF705F93F20CB
:10550000FDF702F912E09DF81F309AB20A4B9A801B
:105510009DF81F309AB2094B9A80094B1B6843F4DF
:105520007F03074A1360034B00221A6009B030BDA5
:10553000046A0008983100206830002010300020F4
:045540009031002086
:1055440000B583B01F4B01221A6001F034FD1E48E0
:1055540001F0DAFF3A20FDF7D5F82020FDF7D2F864
:1055640001F0CFFE03468DF807309DF807303F2B3E
:1055740003D1144B00221A6021E09DF807300A2B56
:1055840003D09DF807300D2B06D13F20FDF7BAF864
:105594000C4B00221A6012E09DF807309AB20B4BB4
:1055A400DA809DF807309AB2094BDA80094B1B6800
:1055B40043F47F03074A1360024B00221A6003B0CE
:1055C4005DF804FB983100207473000868300020F3
:0855D40010300020903100208E
:1055DC0030B5BDB003468DF80730B04B35AC0FCBB2
:1055EC0007C42380AE4B2FAC1D460FCD0FC495E8DE
:1055FC00030020600434218002340B0C2370A94B6F
:10560C0025AC1D460FCD0FC40FCD0FC495E803007C
:10561C00206004342170A44B15AC1D460FCD0FC473
:10562C000FCD0FC40FCD0FC495E80F0007C4237026
:10563C009E4B0EAC1D460FCD0FC495E8070003C45E
:10564C0022809B4B03AC1D460FCD0FC40FCD0FC456
:10565C0095E8070003C42280964B01221A609DF83E
:10566C0007305B005B00944A13443A939DF8073073
:10567C005B005B00914A134439930023ADF8EC3086
:10568C0001F095FC35AB184601F03AFF01F00FFD27
:10569C000346ADF8E230BDF8E230FF2B06D93F20CF
:1056AC00FDF72CF8834B00221A60B0E1BDF8E23014
:1056BC00002B20D13A9B4FF6FF721A803A9B023393
:1056CC004FF6FF721A80399B4FF6FF721A80399B86
:1056DC0002334FF6FF721A809DF807301846FBF71D
:1056EC0013F8774B1B6843F47F03754A1360714BB7
:1056FC0000221A608BE1BDF8E230F52B21D93A9BE0
:10570C009A1C3A92BDF8E2201A803A9B80221A80A9
:10571C00399B9A1C3992BDF8E2201A803A9B1A8860
:10572C00399B1A809DF807301846FAF7EDFF644B49
:10573C001B6843F47F03624A13605E4B00221A60BD
:10574C0065E1BDF8E2300F2B04D8BDF8E2308DF8DE
:10575C00EE3005E0BDF8E230DBB21B098DF8EE301F
:10576C009DF8EE30082B06D83F20FCF7C7FF514BB5
:10577C0000221A604BE19DF8EE300D2B07D9BDF8D5
:10578C00E230F22B03D0BDF8E230F32B6AD19DF856
:10579C00EE300C2B2CD09DF8EE300D2B28D0BDF814
:1057AC00E230F32B24D02FAB184601F0A9FE454B69
:1057BC001B68002B03D0444801F0A2FE02E04348D2
:1057CC0001F09EFE3F20FCF799FF2920FCF796FF85
:1057DC002020FCF793FF00F029F90346ADF8EC30DC
:1057EC00BDF8EC307F2B03D9324B00221A600EE14E
:1057FC0001F0DDFB9DF80730062B03D99DF807302F
:10580C000B2B03D99DF807300E2B07D90EAB18467E
:10581C0001F076FE00238DF8EF3092E025AB1846B0
:10582C0001F06EFE01F0DCFE03468DF8EF309DF8C2
:10583C00EF300A2B0AD09DF8EF300D2B06D03F200D
:10584C00FCF75CFF1B4B00221A60E0E09DF8EF3088
:10585C000A2B03D180238DF8EF3072E000238DF8F2
:10586C00EF306EE09DF8EE300E2B63D10023ADF8D7
:10587C00EC309DF80730062B03D99DF807300B2B25
:10588C0003D99DF807300E2B22D90EAB184601F028
:10589C0037FE00238DF8EF3053E000BF246A000878
:1058AC00346A00084C6A0008746A0008B46A00087C
:1058BC00D06A000898310020743000201C30002081
:1058CC0090310020843100204C67000844670008A8
:1058DC0001F06DFB15AB184601F012FE01F080FED5
:1058EC0003468DF8EF309DF8EF300A2B0ED09DF863
:1058FC00EF300B2B0AD09DF8EF300D2B06D03F204C
:10590C00FCF7FCFE434B00221A6080E09DF8EF3060
:10591C000A2B03D180238DF8EF3012E09DF8EF3085
:10592C000B2B03D181238DF8EF300AE000238DF887
:10593C00EF3006E03F20FCF7E1FE364B00221A6008
:10594C0065E09DF8EF30002B2DD101F030FB03AB5F
:10595C00184601F0D5FD304B1B68002B03D02F48A7
:10596C0001F0CEFD02E02E4801F0CAFD3F20FCF70D
:10597C00C5FE2920FCF7C2FE2020FCF7BFFE00F07C
:10598C0055F803468DF8EF309DF9EF30002B03DB13
:10599C009DF8EF30002B06D13F20FCF7AFFE1D4BDE
:1059AC0000221A6033E09DF8EF301B021AB2BDF9E9
:1059BC00EC3013431BB2ADF8EC303A9B9A1C3A9284
:1059CC00BDF8E2201A803A9BBDF8EC201A80399B76
:1059DC009A1C3992BDF8E2201A803A9B1A88399B9E
:1059EC001A809DF807301846FAF78EFE0D4B9B680F
:1059FC0003F00103002B01D1FBF774FE0A4B1B686B
:105A0C0043F47F03084A1360024B00221A603DB036
:105A1C0030BD00BF98310020843100204C67000855
:0C5A2C0044670008000004509031002086
:105A380000B583B000238DF80730424B1B68002B5C
:105A48002FD0012001F0E9FB03468DF806309DF8C0
:105A58000630EE2B01D1FF2370E09DF806308DF85B
:105A68000730012001F0D9FB03468DF806309DF878
:105A78000630EE2B01D1FF2360E09DF80630FF2BA6
:105A880002D19DF8073059E09DF807301B015AB242
:105A98009DF9063013435BB28DF807309DF8073047
:105AA8004CE001F02CFC03468DF806309DF80630DA
:105AB8003F2B01D1FF2341E09DF806308DF80730D8
:105AC80001F01DFC03468DF806309DF806303F2B8B
:105AD80001D1FF2332E09DF806300D2B02D19DF84D
:105AE80007302BE09DF807301A46920013445B00FC
:105AF800DAB29DF8063013448DF8073001F0FFFB49
:105B080003468DF806309DF806303F2B01D1FF2360
:105B180014E09DF806300D2B02D19DF807300DE0FA
:105B28009DF807301A46920013445B00DAB29DF8DC
:105B3800063013448DF807309DF80730184603B037
:085B48005DF804FB843100202C
:105B500030B5DDB0884B56AC1D460FCD0FC495E86F
:105B6000030084E80300854B51AC1D460FCD0FC4E4
:105B70002B682380824A4FAB92E8030018600433FD
:105B80001970804B44AC1D460FCD0FC40FCD0FC410
:105B900095E8070003C422800234130C23707A4B6B
:105BA00034AC1D460FCD0FC40FCD0FC40FCD0FC4A5
:105BB00095E80F0007C4238002341B0C2370734A3E
:105BC00022AB11464622184601F0DDFB5CABA3F583
:105BD0009C736F4A184611464D231A4601F0D3FBB9
:105BE0005CABA3F5B8736B4A1C4615460FCD0FC4CA
:105BF0000FCD0FC40FCD0FC495E80300206004340F
:105C0000217001F0DAF956AB184601F07FFC01F083
:105C1000D4F92120FCF778FD3A20FCF775FD20200F
:105C2000FCF772FD51AB184601F070FC01F0C5F9AC
:105C30005620FCF769FD3A20FCF766FD2020FCF7B2
:105C400063FD4FAB184601F061FC534801F05EFC68
:105C500001F0B3F94220FCF757FD3A20FCF754FD60
:105C60002020FCF751FD4FAB184601F04FFC4B488C
:105C700001F04CFC01F0A1F94D20FCF745FD3A2064
:105C8000FCF742FD2020FCF73FFD4FAB184601F02A
:105C90003DFC434801F03AFC01F08FF94320FCF74A
:105CA00033FD3A20FCF730FD2020FCF72DFD4FABF3
:105CB000184601F02BFC3B4801F028FC01F07DF96F
:105CC0004820FCF721FD3A20FCF71EFD2020FCF7C0
:105CD0001BFD4FAB184601F019FC334801F016FCD0
:105CE00001F06BF94420FCF70FFD3A20FCF70CFDA6
:105CF0002020FCF709FD4FAB184601F007FC2B48AC
:105D000001F004FC2A4801F001FC01F056F958208A
:105D1000FCF7FAFC3A20FCF7F7FC2020FCF7F4FC37
:105D20004FAB184601F0F2FB204801F0EFFB214891
:105D300001F0ECFB01F041F944AB184601F0E6FB41
:105D400001F03BF934AB184601F0E0FB01F035F906
:105D500022AB184601F0DAFB01F02FF90EAB184622
:105D600001F0D4FB01F029F96B46184601F0CEFB97
:105D700000BF5DB030BD00BFFC6A0008146B0008B6
:105D8000286B0008306B00085C6B00089C6B0008F7
:105D9000E46B0008346C0008E4720008E866000850
:105DA00014670008A06F00087473000838670008C3
:085DB000446700084C6700087D
:105DB80030B5BDB0A74B2FAC1D460FCD0FC40FCDCE
:105DC8000FC42B681A46228002341B0C2370A24B86
:105DD80026AC1D460FCD0FC40FCD0FC42B68237002
:105DE8009E4B20AC1D460FCD0FC495E803002060E4
:105DF8000434218002340B0C2370994B1BAC1D46D4
:105E08000FCD0FC42B682370964A19AB92E8030094
:105E180083E80300944B12AC1D460FCD0FC495E8E0
:105E2800070003C42270914B0BAC1D460FCD0FC465
:105E380095E8070003C422808D4A08AB07CA03C34C
:105E48001A708C4A05AB07CA03C31A808A4B01AC87
:105E58000FCB84E80F0001F0ACF8884801F052FB42
:105E680001F0A7F85620FCF74BFC3A20FCF748FC59
:105E78002020FCF745FC19AB184601F043FB80488D
:105E880001F040FB3A20FCF73BFC2020FCF738FCF3
:105E98007C4B1A897B4B5B8913409BB24FF6FF7290
:105EA800934204D140F28343ADF8EE300CE0754BD9
:105EB8001B891B021AB2734B5B891BB2DBB21BB284
:105EC80013431BB2ADF8EE30BDF8EE30184601F0C2
:105ED800D7FA2F20FCF714FC2020FCF711FC694BA3
:105EE8009A89684BDB8913409BB24FF6FF72934245
:105EF80004D145F24073ADF8EE300CE0614B9B895C
:105F08001B021AB25F4BDB891BB2DBB21BB2134315
:105F18001BB2ADF8EE30BDF8EE30184601F0B0FA1D
:105F2800594B1B6803F0FF23B3F57F4F2AD101F0CB
:105F380040F826AB184601F0E5FA544B1B891B02C2
:105F48001AB2524B5B891BB2DBB21BB213431BB2B2
:105F5800ADF8EE30BDF8EE30184601F091FA4B4B33
:105F68009B891B021AB2494BDB891BB2DBB21BB2FD
:105F780013431BB2ADF8EE30BDF8EE30184601F011
:105F88007FFA30E0404B1B6803F0FF23B3F1FF2F8B
:105F980029D101F00EF82FAB184601F0B3FA3B4BAC
:105FA8001B891B021AB2394B5B891BB2DBB21BB2CD
:105FB80013431BB2ADF8EE30BDF8EE30184601F0D1
:105FC8005FFA324B9B891B021AB2304BDB891BB23A
:105FD800DBB21BB213431BB2ADF8EE30BDF8EE30A6
:105FE800184601F04DFA00F0E4FF4220FCF788FB68
:105FF8003A20FCF785FB2020FCF782FB19AB1846FA
:1060080001F080FA224801F07DFA3A20FCF778FB8B
:106018002020FCF775FB1B4B1B888DF8ED309DF895
:10602800ED30184600F02EFA174B1B6823F47F0357
:1060380023F47F43FF2B2DD100F0BBFF26AB18467E
:1060480001F060FA114B1B88DBB2184600F01AFA0F
:1060580035E000BF6C6C0008906C0008B46C000858
:10606800CC6C0008E06C0008E86C0008046D0008BF
:10607800206D00082C6D0008386D00082474000895
:10608800E4720008103000209031002068300020B1
:10609800E8660008AC4B1B6823F47F0323F47F43B6
:1060A800AA4A93420BD100F084FF2FAB184601F0A7
:1060B80029FAA74B1B88DBB2184600F0E3F900F079
:1060C80078FF4D20FCF71CFB3A20FCF719FB202039
:1060D800FCF716FB9F4801F015FA3A20FCF710FB75
:1060E8002020FCF70DFB9C4B5B884FF6FF72934218
:1060F80003D11F238DF8ED3003E0974B5B888DF8B3
:10610800ED309DF8ED30184600F0BCF900F051FF75
:106118004320FCF7F5FA3A20FCF7F2FA2020FCF7C6
:10612800EFFA8E4801F0EEF93A20FCF7E9FA202060
:10613800FCF7E6FA884B9B884FF6FF72934203D12F
:1061480001238DF8ED3005E0834B9B88DBB20133EA
:106158008DF8ED309DF8ED309BB21846FCF72AFB20
:1061680000F027FF4820FCF7CBFA3A20FCF7C8FAE2
:106178002020FCF7C5FA7A4801F0C4F93A20FCF768
:10618800BFFA2020FCF7BCFA734BDB884FF6FF728E
:10619800934203D102238DF8ED3003E06E4BDB8888
:1061A8008DF8ED309DF8ED303033DBB21846FCF752
:1061B800A7FA00F0FEFE6B4801F0A4F96A4B1B68D1
:1061C800002B03D1694801F09DF902E0684801F00D
:1061D80099F900F0EEFE20AB184601F093F900F0B3
:1061E800E8FE01238DF8EC3040E19DF8EC305B00CF
:1061F8005B00604A13443993399B02333893399BC7
:106208001B880F2B12D8399B1B888DF8EA309DF814
:10621800EA301B015BB223F00F035AB24E4B9B8846
:106228005BB213435BB28DF8E9300CE0399B1B88F5
:106238001B099BB2DBB203F00F038DF8EA30399BE0
:106248001B888DF8E9309DF8EC305A1E1346DB00A8
:106258009B1A5B00484A1344184601F053F9399BCE
:106268001A88389B1B8813409BB24FF6FF729342E3
:1062780003D1424801F046F9EDE01BAB184601F0A6
:1062880041F99DF8E930184600F099FD9DF8E9308C
:10629800F32B00F2CC809DF8E930F22B03D09DF867
:1062A800EA300B2B39D8304B1B68002B14D0389BA5
:1062B8001B88DBB203F07F03DBB2184600F07FFDDA
:1062C800389B1B881B0A9BB2DBB203F07F03DBB24F
:1062D800184600F074FD11E0389B1B8803F07F031B
:1062E8009BB21846FCF766FA389B1B881B0A9BB2C0
:1062F80003F07F039BB21846FCF75CFA389B1B88B7
:106308001BB2002B04DB0BAB184601F0FBF8A2E034
:1063180008AB184601F0F6F89DE09DF8EA300E2B20
:1063280059D1114B1B68002B2AD0389B1B88DBB234
:10633800184600F044FD389B1B881B0A9BB2DBB251
:10634800184600F03CFD29E090310020FF0000FFD6
:10635800683000201467000810300020A06F000883
:106368007473000838670008843100204467000807
:106378004C6700081C300020CC6F000834740008FB
:10638800389B1B88DBB29BB21846FCF713FA389B84
:106398001B881B0A9BB21846FCF70CFA389B1B8813
:1063A80003F47F43B3F5014F04D105AB184601F060
:1063B800A9F850E0389B1B8803F47F43B3F5004FDE
:1063C80004D108AB184601F09DF844E00BAB184621
:1063D80001F098F83FE02A4B1B68002B08D0389B47
:1063E8001B881B0A9BB2DBB2184600F0E8FC06E0EB
:1063F800389B1B881B0A9BB21846FCF7DBF9202048
:10640800FCF77EF92020FCF77BF92020FCF778F9CF
:10641800389B1B881BB2002B04DB12AB184601F01B
:1064280071F818E008AB184601F06CF813E0002387
:106438008DF8EB3007E02020FCF762F99DF8EB308F
:1064480001338DF8EB309DF8EB30062BF3D901AB17
:10645800184601F057F89DF8EC30112B01D000F0E8
:10646800A8FD9DF8EC3001338DF8EC309DF8EC3048
:10647800112B7FF6BAAE00BF00BF3DB030BD00BFE4
:04648800843100203B
:10648C0000B583B003468DF807309DF80730644A99
:10649C00A2FB0323DB08DBB23033DBB21846FCF77C
:1064AC002DF99DF807205E4BA3FB0213D9080B4670
:1064BC009B000B445B00D31ADBB23033DBB21846C3
:1064CC00FCF71CF99DF80730602B00F08B80602BDB
:1064DC0000F39580262B41DC0B2BC0F290800B3BFC
:1064EC001B2B00F28C8001A252F823F06F65000880
:1064FC000B6600080B6600080B6600080B660008AC
:10650C000B6600080B6600080B660008896500081E
:10651C000B6600080B6600080B6600080B6600088B
:10652C000B6600080B6600080B6600080B6600087B
:10653C000B6600080B6600080B660008A3650008D4
:10654C000B6600080B6600080B6600080B6600085B
:10655C000B6600080B660008BD650008392B34D0AB
:10656C004DE03520FCF7CAF83220FCF7C7F8302094
:10657C00FCF7C4F83020FCF7C1F84DE03220FCF7F2
:10658C00BDF83020FCF7BAF83020FCF7B7F8202023
:10659C00FCF7B4F840E04D20FCF7B0F84920FCF7CC
:1065AC00ADF84420FCF7AAF84920FCF7A7F833E033
:1065BC003420FCF7A3F83020FCF7A0F83020FCF7CF
:1065CC009DF82020FCF79AF826E03620FCF796F888
:1065DC003020FCF793F83020FCF790F82020FCF7E3
:1065EC008DF819E03020FCF789F83020FCF786F89C
:1065FC002020FCF783F82020FCF780F80CE03F20EB
:10660C00FCF77CF83F20FCF779F83F20FCF776F894
:10661C002020FCF773F800BF00BF03B05DF804FB4B
:04662C00CDCCCCCC39
:10663000114B1B68104A43F0010313600E4B0022FC
:106640009A600D4B1B680C4A23F0A85323F41023C7
:106650001360094B4FF48052DA60074B1B68064AFF
:1066600023F480231360044B00229A61034B4FF004
:1066700000629A6000BF70470010024000ED00E029
:1066800082B001900A4B1B68002B0DDA084B1B6887
:10669000074A43F000431360019B18331A68019BBB
:1066A000183302321A6000E0FEE702B0704700BF04
:0466B0002CED00E0ED
:1066B40020286329323031362D323120572E53634E
:0866C40068656D6D65727400DC
:0466CC0004030904B6
:1066D00018035500530042002D004D00690064006E
:0866E000690043006F006D002A
:1066E80053657269616C20434F4D20426175647235
:1066F800617465202861637469766520696E20522B
:0C670800532D323332204D6F64652900A0
:106714004D49444920426175647261746520286161
:10672400637469766520696E204D494449204D6F34
:04673400646529006F
:0C6738004E756D626572426173653D0034
:08674400646563696D616C007E
:04674C006865780004
:10675000FEE7FEE7FEE7FEE7FEE7FEE7FEE7FEE711
:10676000FEE7FEE7FEE7FEE7FEE7FEE7FEE7FEE701
:10677000FEE7FEE7FEE7FEE7FEE7FEE7FEE7FEE7F1
:10678000FEE7FEE7FEE7FEE7FEE7FEE7FEE7FEE7E1
:10679000FEE7FEE7FEE7FEE7FEE7FEE7FEE7FEE7D1
:1067A000FEE7FEE7FEE7FEE7FEE7FEE7FEE7FEE7C1
:1067B000FEE7FEE7FEE7FEE7FEE7FEE7FEE7FEE7B1
:1067C000FEE7FEE7FEE7FEE7FEE7FEE7FEE7FEE7A1
:1067D000FEE7FEE7FEE7FEE7FEE7FEE7FEE7FEE791
:1067E000FEE7FEE7FEE7FEE7FEE7FEE7FEE7FEE781
:1067F000FEE7FEE7FEE7FEE7FEE7FEE7FEE7FEE771
:10680000FEE7FEE7FEE703488546FFF711FF00F0CD
:0868100003B87047008001206D
:1068180011488546114C20680434004201D0804755
:10682800F9E70F480F49091A082903DB002202601B
:10683800043001600C480D49884205D002680430D4
:1068480003B4904703BCF7E700208646EC460020D7
:106858000021074A9047FEE70080012014760008CF
:10686800C0310020C03500202172000821720008C4
:046878004D020008C5
:10687C001EF0040F0CBFEFF30880EFF30980014901
:08688C000847000081660008C6
:10689400536574757020686173206368616E676501
:1068A400642E2053617665207769746820277C27DD
:1068B40020666F72207065726D616E656E742073F0
:1068C400746F7261676520696E20466C617368003D
:1068D4002020202020202043616E63656C204578B1
:1068E40069742077697468203C4553433E00000076
:1068F4005361766520746F20466C6173683F202D68
:106904003E7479706520616761696E200000000043
:10691400204E4F542053415645442120000000008E
:106924002052656C6F6164205365747570206672C3
:106934006F6D20466C6173683F202D3E74797065DD
:1069440020616761696E2000204E4F542052454CEF
:106954004F41444544212000436F6E6669672049D6
:106964006E7075742320000020656E746572206E4D
:1069740065772056696420283420686578206E691C
:1069840062626C6573293A200000000020656E7411
:106994006572206E6577205069642028342068650C
:1069A40078206E6962626C6573293A2000000000E9
:1069B400434F4D20626175642072617465202D20FF
:1069C400656E74657220666972737420322064691E
:1069D400676974733A2000004D4944492062617527
:1069E400642072617465202D20656E746572206662
:1069F400697273742032206469676974733A200081
:106A0400456E746572204D494449206368616E6E19
:106A1400656C2028312E2E2E3136293A20000000B4
:106A240053746174757328686578293F20000000E9
:106A3400202D3E317374204D4944492064617461B2
:106A440020627974652800002020506F72742052EF
:106A54006561643A2744273D6469676974616C2CF5
:106A64002741273D616E616C6F673F200000000085
:106A74002020506F727420526561643A2744273D88
:106A84006469676974616C2C2741273D616E616C90
:106A94006F672837626974292C2742273D616E612C
:106AA4006C6F67283132626974293F20000000004E
:106AB4002020506F727420526561643A20646967C3
:106AC4006974616C206F6E6C7900000020206C6129
:106AD4007374204D4944492064617461206279745F
:106AE40065207768656E20627574746F6E207075AA
:106AF40073686564280000004C697374206F662015
:106B0400536574757020436F6D6D616E64733A00E4
:106B14006C6973742041637475616C20536574757A
:106B2400700000007365742000000000312C322CCA
:106B3400332C342C352C362C372C382C392C313042
:106B44002C31312C31322C31332C31342C312C3149
:106B54002C31362C553A0000202020736574204DCA
:106B6400494449206D7367732072656C6561736570
:106B740064206279206368616E6765206F662049CE
:106B84002F4F206E6F20312E2E39202B55736572B6
:106B9400427574746F6E0000403A2072656C6F61C8
:106BA400642073657475702066726F6D20466C6125
:106BB400736820286368616E6765732073696E6308
:106BC40065206C61737420506F7765725570206115
:106BD40072652063616E63656C6C656429000000F6
:106BE4007C3A2073617665206E65772073657475D1
:106BF40070207065726D616E656E746C7920696E5B
:106C040020466C617368202877696C6C2062656328
:106C14006F6D6520616374697665206174206E65AB
:106C2400787420506F776572205570290000000039
:106C3400453A20657869742053455455502C207288
:106C4400657475726E20746F20626964697265631D
:106C540074696F6E616C20636F6D6D756E696361CD
:106C640074696F6E0000000020202020202028730B
:106C7400617665642C206E6F74207965742061637D
:106C8400746976652C206E65773A000020202020F8
:106C94002020286D6F6469666965642C206E6F74AA
:106CA4002073617665642C206E65773A00000000DD
:106CB400496E707574204368616E6765206D6573F5
:106CC40073616765733A000020636F6E6669677568
:106CD400726564206D736720000000004163747561
:106CE400616C2000204469673A73656E64206461B6
:106CF4007461206966207075736865640000000023
:106D0400204469673A73656E64206461746132205B
:106D140069662070757368656400000020416E61C7
:106D2400376269740000000020416E61313262698B
:106D34007400000053696E676C6520627974652085
:046D44006D73670004
:0E6D48005553422D4D696469436F6D207600EE
:106D560000B583B00123019305E00198F9F7D7FC4C
:106D6600019B01330193019B112BF6D900BF00BF94
:066D760003B05DF804FB10
:106D7C00120110010200004083044057060300007A
:026D8C00000104
:106D8E0000B583B003468DF807309DF807301846DE
:106D9E00FBF79DFC9DF807301846FDF744FA00BF3F
:066DAE0003B05DF804FBD8
:106DB400120368006F006D0065006D0061006400DF
:026DC400650068
:106DC60000B585B003468DF807309DF807301B09DE
:106DD6008DF80F309DF80F3030338DF80F309DF859
:106DE6000F30392B04D99DF80F3007338DF80F304B
:106DF6009DF80F301846FBF784FC9DF8073003F02A
:106E06000F038DF80F309DF80F3030338DF80F30AB
:106E16009DF80F30392B04D99DF80F3007338DF8C4
:106E26000F309DF80F301846FBF76BFC2020FBF760
:0A6E360068FC00BF05B05DF804FB26
:026E4000000050
:106E420000B585B00346ADF80630BDF80630B3F59F
:106E5200805F03D340F6FF73ADF80630BDF806300D
:106E62001B0A9BB2DBB203F00F038DF80F309DF8C3
:106E72000F301846FBF76DFCBDF806301B099BB2BC
:106E8200DBB203F00F038DF80F309DF80F30184678
:106E9200FBF75FFCBDF80630DBB203F00F038DF8A1
:106EA2000F309DF80F301846FBF753FC2020FBF7FC
:0A6EB2002AFC00BF05B05DF804FBE8
:106EBC001201000200000040830442570603020145
:026ECC000001C3
:106ECE0000B585B00190019B1B0FDBB203F00F03E1
:106EDE008DF80F309DF80F30184600F0B2FA019B76
:106EEE001B0EDBB203F00F038DF80F309DF80F3041
:106EFE00184600F0A6FA019B1B0DDBB203F00F0340
:106F0E008DF80F309DF80F30184600F09AFA019B5D
:106F1E001B0CDBB203F00F038DF80F309DF80F3012
:106F2E00184600F08EFA019B1B0BDBB203F00F0329
:106F3E008DF80F309DF80F30184600F082FA019B45
:106F4E001B0ADBB203F00F038DF80F309DF80F30E4
:106F5E00184600F076FA019B1B09DBB203F00F0313
:106F6E008DF80F309DF80F30184600F06AFA019B2D
:106F7E00DBB203F00F038DF80F309DF80F3018467B
:106F8E0000F05FFA2020FBF7A2FB00BF05B05DF812
:026F9E0004FBF2
:106FA000476C6F62616C204D494449204368616EB3
:0A6FB0006E656C28312D3136290082
:106FBA0008B50D20FBF7A3FB0A20FBF7A0FB00BFD7
:026FCA0008BD00
:106FCC00496E707574312028504132293A00496E4F
:106FDC00707574322028504133293A00496E70750F
:106FEC0074332028504230293A00496E707574343D
:106FFC002028504134293A00496E70757435202888
:10700C00504131293A00496E707574362028504130
:10701C0030293A00496E7075743728504131352942
:10702C003A00496E707574382028504237293A005E
:10703C00496E707574392028504233293A00496ED4
:10704C00707574313028504235293A00496E70758C
:10705C0074313128504234293A00496E70757431BC
:10706C003228504137293A00496E707574313328F3
:10707C00504136293A00496E7075743134285041AC
:10708C0035293A00496E70757431352850423929CA
:10709C003A00496E707574313628504238293A00DE
:0E70AC00496E707574552850433133293A00EF
:1070BA0000B583B00023ADF80630012000F0ACF82B
:1070CA0003468DF805309DF80530ED2B02D94FF4B3
:1070DA007F436AE09DF805309BB21B01ADF806308C
:1070EA00012000F099F803468DF805309DF8053027
:1070FA00EE2B02D14FF47F4357E09DF80530FF2B6A
:10710A0019D1BDF80630002B02D1BDF806304CE08B
:10711A00BDF806301B09ADF80630BDF80630082B5D
:10712A0003D9BDF806300E2B02D94FF47F433CE059
:10713A00BDF8063039E09DF805309AB2BDF8063040
:10714A001343ADF80630BDF80630002B02D1BDF866
:10715A0006302AE0BDF806308F2B02D84FF47F4361
:10716A0023E0BDF80630F02B03D0BDF80630F72B2C
:10717A0002D14FF47F4318E0BDF80630F12B0FD04F
:10718A00BDF80630F42B0BD0BDF80630F52B07D02E
:10719A00BDF80630F92B03D0BDF80630FD2B02D11D
:1071AA004FF47F4301E0BDF80630184603B05DF89E
:0271BA0004FBD4
:1071BC000902650002010080310904000000010190
:1071CC000000092401000109000101090401000269
:1071DC000103000007240100014100062402010103
:1071EC00000624020202000924030103010201002B
:1071FC000924030204010101000905810240000079
:10720C0000000525010103090502024000000000F1
:05721C00052501010140
:1072220000B585B003468DF8073000BFFBF787FB3A
:107232000346ADF80C30BDF80C30002BF6D0BDF88B
:107242000C308DF80F309DF80730002B09D09DF8D7
:107252000F300A2B03D09DF80F300D2B01D1FF23E5
:107262003BE09DF80F303F2B04D13F20FBF74BFA58
:10727200EE2332E09DF80F30602B08D99DF80F30D5
:107282007A2B04D89DF80F30203B8DF80F309DF8F3
:107292000F30402B08D99DF80F30462B04D89DF8AB
:1072A2000F30073B8DF80F309DF80F302F2B10D980
:1072B2009DF80F303F2B0CD89DF80F30303B8DF8E6
:1072C2000F309DF80F301846FBF743FA9DF80F3048
:1072D20003E03F20FBF717FAEE23184605B05DF8EE
:0272E20004FBAB
:1072E400555342205669642F506964206F66207498
:1072F4006869732064657669636520286865782900
:017304000088
:1073060000B583B000BFFBF718FB0346ADF80630A7
:10731600BDF80630002BF6D0BDF806308DF80530E6
:107326009DF805300A2B03D09DF805300D2B01D1B1
:107336000D2318E09DF805302F2B03D99DF8053055
:10734600392B04D93F20FBF7DCF93F230BE09DF8EE
:1073560005301846FBF7D5F99DF80530303B8DF81A
:0E73660005309DF80530184603B05DF804FBB5
:107374004879737465726573697328302E2E3929C0
:017384000008
:10738600844640EA010313F0030F18D18446202AED
:107396000BD32DE9F007B1E8F807A0E8F807A2F14A
:1073A6002002202AF7D2BDE8F007042A07D351F8B5
:1073B600043B40F8043BA2F10402042AF7D2002A57
:1073C60005D011F8013B00F8013B013AF9D16046BE
:0273D6007047FE
:1073D8000902430002010080310904000001020291
:1073E80000000524001001052401030004240207FD
:1073F8000524060001070583031000400904010065
:10740800020A000000070581024000010705020288
:0374180040000130
:07741C0000C201000000089E
:0F742400436F6E66696775726174696F6E3A00C7
:10743400204E4F206D736720636F6E6669677572A7
:037444006564007C
:077448004572726F723A00F9
:1074500000B585B003468DF807309DF8073030330E
:107460008DF80F309DF80F30392B04D99DF80F306F
:1074700007338DF80F309DF80F301846FBF72EF9C3
:0874800000BF05B05DF804FB3C
:1074880000B585B00346ADF80630BDF806301B0BD5
:107498009BB2DBB203F00F038DF80F309DF80F306D
:1074A8001846FBF753F9BDF806301B0A9BB2DBB24E
:1074B80003F00F038DF80F309DF80F301846FBF7D7
:1074C80045F9BDF806301B099BB2DBB203F00F0388
:1074D8008DF80F309DF80F301846FBF737F9BDF8D7
:1074E8000630DBB203F00F038DF80F309DF80F3034
:1074F8001846FBF72BF92020FBF702F900BF05B06F
:047508005DF804FB2B
:10750C0000B585B0019004E09DF80F301846FBF7EC
:10751C00F5F8019B5A1C01921B788DF80F309DF8E1
:10752C000F30002BF0D100BF00BF05B05DF804FB9D
:10753C0000B583B04FF0A0435A694FF0A0439B694C
:10754C0013400193019B002B46D0019B03F40023B5
:10755C00002B01D0FCF796F8019B03F48023002B41
:10756C0001D0FBF7CBFE019B03F01003002B01D0E5
:10757C00FBF76AFD019B03F00803002B03D04FF0CF
:10758C00A04308225A61019B03F48053002B06D0C0
:10759C00FBF7FAFB4FF0A0434FF480525A61019B6A
:1075AC0003F40053002B04D04FF0A0434FF40052CF
:1075BC005A61019B002B04DA4FF0A0434FF00042BC
:1075CC005A61019B03F40063002B06D04FF0A043DB
:1075DC004FF400625A6100E000BF03B05DF804FB99
:1075EC0000B583B00120FFF716FE03468DF8073077
:1075FC009DF80730EE2B01D1FF2301E09DF80730F9
:08760C00184603B05DF804FB11
:107614004576000810000020AB3100005B760008BE
:107624000000002034760008100000000000000074
:107634000E1000200E2000200E30002000093D0016
:10764400206861680834094204D0002202700130C5
:067654000139FBD1704773
:10765A0020686168A2680C34124205D00B78037066
:0A766A0001300131013AF9D17047F7
:040000050800680780
:00000001FF
